:020000040800F2
:10000000601E0020D5000008DD000008DF000008A9
:1000100000000000000000000000000000000000E0
:10002000000000000000000000000000E1000008E7
:100030000000000000000000E3000008255900084F
:1000400000000000E7000008E7000008BB400008CF
:10005000E7000008E7000008FD1600083517000853
:100060006D1700084D13000881130008B513000830
:10007000E70000082565000895400008E700000833
:10008000E7000008E700000845090008E70000084D
:10009000B564000891650008D5640008E700000811
:1000A000E7000008E70000081D320008756400083A
:1000B0009564000801320008E7000008E700000826
:1000C0000348854600F0E6FB00480047DD7900085C
:1000D000601E00200448804704480047FEE7FEE712
:1000E000FEE7FEE7FEE7FEE7C15A0008C100000890
:1000F000F0B51FB40646002082B0054640240191A9
:1001000000901BE0019922460F46304600F0FDFAB0
:10011000049A059B801A994110D31046194622462D
:1001200000F0E3FA361A8F410197224601200021A0
:10013000009F00F0DAFA38184D4100902046641E06
:100140000028DFDC019B00982946324607B0F0BD4D
:1001500030B5434351435C18010C130C0D465D430D
:100160002C1980B292B20546554351430A0C09043A
:100170004D1962415843010C00044019514130BDF2
:1001800010B5431A934209D28318881803E0401E21
:1001900001785B1E1970521EF9D210BD03460B4345
:1001A0009B0703D009E008C9121F08C0042AFAD22D
:1001B00003E00B780370401C491C521EF9D210BD9D
:1001C000D2B201E00270401C491EFBD270470022EF
:1001D000F6E710B513460A4604461946FFF7F0FF46
:1001E000204610BD421C0178401C0029FBD1801A1A
:1001F000704730B504460020034600E05B1C934284
:1002000003D2E05CCD5C401BF8D030BD70B5024637
:100210004A40D50F40004A00ED0740085208002828
:1002200014D0002A12D0C40DD30D41020120C00504
:100230005202490A520AE41A091812187D349142EE
:1002400001D3641C00E04900002C01DA002070BDDD
:100250000023914201D3891A034340084900002832
:10026000F7D100290AD0914202D10121C90705E046
:10027000914201D2012101E00121C943E005C018EA
:10028000401900F066FA70BDF0B5074608465840C0
:1002900087B0C00F049048000E4659004008490836
:1002A000BC1A884105D2384631461E4617460B46D1
:1002B00002465800400810434CD0300D03904005D2
:1002C0005900400D490D0590401A0290402872DAFD
:1002D00018030121000B09050843019004980092BE
:1002E000002805D0019952420020884100920190D7
:1002F000029840210A1A0199009800F0F6F9054683
:100300000C466B4607CB00F011FAC0197141039AF5
:100310000E0D0023D71756401A467A40164344D094
:10032000049A002A2DD0029A012A039A15DC12059C
:10033000C01A914101263605001C7141D20F059E5D
:10034000D2070093019202962A46234600F04FFA04
:1003500007B0F0BD38463146FAE71605224A0F4687
:10036000B218C01AB74101210905001C4F410018FD
:100370007F41114618187941E20F10436D1964410D
:1003800013E0E2076D0815436408C2071443039A9B
:1003900001261205C01A91413605001C7141CE0795
:1003A000400830434908C01851412A46234600F00E
:1003B00011FACDE7FFE7049801224000C117121A95
:1003C00000238B4104983146C417381AA141EEE747
:1003D00030B40124E407634030BC55E730B4012455
:1003E000E407614030BC4FE70000E0FFF0B51FB408
:1003F00088B00B990998002448400999C00F49001A
:1004000049080991C0070B990090490049080B91D0
:1004100009990898A64608431CD00B990A980843E6
:1004200018D0099801244000420D4800410D099858
:1004300024050003000B204309900B980003000BD8
:1004400020430B9050181C4940180022019014467C
:10045000104605E0002001460DB0F0BD032801DA8A
:10046000034600E003239C46C11A0AAE0AE05F007F
:1004700008ADED5B4F00F75B7D430027AA187C4178
:10048000491C5B1E6145F2DD410004AB5A52210458
:10049000120C0A43240C401C0828DFDB0198029050
:1004A0000099704601910090059B049A079906985F
:1004B00000F09DF9D0E700000DFCFFFFF0B50C4601
:1004C0005C4085B0E40FE40703944C000026640808
:1004D00059009446490802460296224321D06246BA
:1004E0000A431ED06200570D4A000E032303550D28
:1004F000012402462C492405781B1B0B360B40189F
:1005000023432643614600901C46501AB44103D34E
:100510000098401C009002E0921800985B4100286F
:1005200003DA0020014605B0F0BD002001210905D5
:100530000746864611E064461D46141BB54106D3A6
:100540006546521BB341744607430C43A646CD078C
:1005500040084908284392185B4105460D43EAD1FB
:100560001046184313D06046194650407140084366
:1005700006D06046101AB34106D20122002306E0DD
:1005800000220123DB0702E00122D243531000982E
:1005900074460105381C6141029C039D00196941A4
:1005A00000F018F9BFE70000FD030000C217C10FFB
:1005B000504010B54018CA079623002100F0D1F82A
:1005C00010BD10B500229623114600F0CAF810BDE8
:1005D0000EB505490291002100910A460B46019192
:1005E00000F005F903B000BD330400000EB5054A64
:1005F0000292002200921346019200F0F8F803B034
:1006000000BD0000330400004A0009030123090B68
:100610001B051943094B10B5520D9A4201DA00200F
:1006200010BD064B34339A4203DC9A1A00F06DF881
:1006300010BD03495118884010BD0000FF030000A1
:10064000CDFBFFFF4A0009030123090B1B051943DA
:100650000A4B10B5520D9A4202DA0020014610BD35
:10066000064B34339A4203DC9A1A00F04EF810BD60
:10067000034BD21800F039F810BD0000FF03000052
:10068000CDFBFFFFC20FD207400040080BD0C10DC9
:100690000723DB01C91840020905400A1143C208BB
:1006A00040071143704700200146704770B504466B
:1006B000002903D000202022012310E0002801D0CF
:1006C0000020C043C046C0460DE02546D5408D42BF
:1006D00005D30D469540641B1D46954040191546AF
:1006E000521E002DF1DC214670BD10B5202A04DB1E
:1006F0000146203A9140002010BD914020239C1AD1
:100700000346E3401943904010BD10B5202A04DB96
:100710000846203AD040002110BD0B46D340D040BF
:100720002024A21A91400843194610BD10B5202A72
:1007300006DBCB170846203A1041C1170B4306E0F1
:100740000B461341D0402024A21A91400843194679
:1007500010BD002904DA401C490001D140084000C6
:10076000704770B40024050C05D11024000402D198
:10077000002921D01124050E01D100020834050FF3
:1007800001D10001241D850F01D18000A41C002887
:1007900001DB4000641C002908D020252E1B0D46DB
:1007A000F540A14000D001212943084301061B1B4D
:1007B000000ADB1D02D5002070BC7047DB0518184D
:1007C00080180029F8DA401C4900F5D170BC4008B7
:1007D0004000704710B5002B08DA0024401C61412E
:1007E00092185B411A4301D14008400010BDF0B59A
:1007F0001FB482B005460C0003D0084607F02AF962
:1008000002E007F027F920300246009021462846F2
:10081000FFF76BFF049B059A04460F4618431143EC
:10082000084314D0184610431BD0009840210A1AE0
:1008300018460599FFF769FF05460E46009A059987
:100840000498FFF752FF084305D0012004E020463A
:10085000394607B0F0BD0020C11705430E432C43B5
:10086000374300990E986305401A7905E40A00227F
:100870000C43FD0A0A3002D500200146E9E70105D4
:10088000101969410C9C0D9D00196941FFF7A2FFE9
:10089000DFE70000064C0125064E05E0E36807CCC3
:1008A0002B430C3C98471034B442F7D3FFF70CFCB1
:1008B0000899000828990008F0B585B00D4606464D
:1008C00001A800248470048002F046FB280C01AFCC
:1008D00078713E71300CF870300AB870BC72FF202D
:1008E0000090023038810124FC803C801248049042
:1008F0002046394601F0B6FD300E3871280AF870EE
:10090000BD700220394601F0ADFD204601F022FE07
:1009100020462146224601F08BFDA00407490860CD
:100920000098000406490A6882430A60204601F0E4
:100930001DFE05B0F0BDC04600401C4500E100E0D2
:1009400010E400E010B50120010301F063FD01286F
:1009500014D10B4CE079002801D0401EE071012039
:1009600000F010F8E1680818E060022000F00AF8D2
:10097000216908182061607A401C607210BDC04671
:100980001411002080B582B000210191012800D00F
:10099000022001F037FD01900120C0030199090AEE
:1009A000081880B201990190019802B080BD000042
:1009B000B0B50120C403A72003252946224603F031
:1009C000F9FE05490880AA202946224603F0F2FED6
:1009D00002490880B0BDC046D60C0020D40C0020CF
:1009E000B548016901220A70016942224A70016911
:1009F0000C228A7002690021D17002693A231371B6
:100A00000269517102693C2393710269D1710269D3
:100A10003E2313720269517202693723937202698D
:100A2000D172026950231373026951730269512311
:100A300093730269D173016990220A7401690E22CD
:100A40008A70112141817047F0B584B09A490869D4
:100A50000122027008692B23437008690E238370FA
:100A60000869C270086902710869FF234371086947
:100A700005238371086903230393C3710869002365
:100A80000193037208690D2302934372086953238B
:100A9000837208694923C372086941230373086993
:100AA0005223437308694723837308694F23C37331
:100AB00008692D23037408695623837208694D233E
:100AC000C3720869312300930373086930234373A9
:100AD000086983730869C3730E690C233376022790
:100AE000F7757748057875764578B5768578F57623
:100AF000C5783577057975774579B5778579F5774F
:100B0000C579202435552036047A7470447AB4703F
:100B1000847AF470C07A019D3574F2730424B4733E
:100B200075733273039AF272029AB27273720B2265
:100B300032720A22F271B471777130710098488173
:100B400004B0F0BD10B55C48016901220A7001696A
:100B500043224A7002691221917003690022DA70FF
:100B6000036983241C7103695A71036985249C718C
:100B70000369DA7103698B241C7203695A72036971
:100B800096249C720369DA72036998241C730369C2
:100B90005A7303699A249C730369DA7303699C246A
:100BA0001C7403695A740369F2249C740369DA742F
:100BB00002699170F02111751521418110BDC04667
:100BC00080B500F001F880BDF0B5CDB04BAE00248B
:100BD000B471FF200230B08034484B90344D284629
:100BE000314601F0DBFFB47101273802B080314893
:100BF0004B902846314601F0D1FF08212846224675
:100C000002F057F8102128463A4602F052F87D20AB
:100C1000C00006F0ACFE284928A0486103204881A6
:100C200004F028FD0A2006F0A2FE641C642CF9D111
:100C3000234881780A9141780991C17804794679ED
:100C40008779C579027A437A807A00910194029675
:100C5000039704950592069307900BAC19A12046C3
:100C6000099A0A9B06F0E2FE2046FFF7BBFA010450
:100C7000114D04D00BA96961688104F0FBFC0024CC
:100C80000A2006F074FE641C642CF9D118A0686177
:100C90000920688104F0EEFC00240A2006F067FEBB
:100CA000641C642CF9D14DB0F0BDC04608000100B1
:100CB0000008014010000100A40100202B2B2B0094
:100CC0000100002041542B4E414D453D312C353320
:100CD00034393431353225782578257825782578CA
:100CE000257825782578257825780D0A00000000DC
:100CF00041542B455849540D0A000000B0B582B04C
:100D0000044601A90020887001250D80064801F0E5
:100D10004BFC2846214601F0C7FC2846294601F035
:100D20007FFC02B0B0BDC04600A402407047000086
:100D30000248017801220A4302707047B20D002078
:100D400010B50122012804D0022809D19405064AD1
:100D500001E01405034A116001F04EFC03480460F1
:100D600010BDC046100D0020140D002000E100E071
:100D700010B500290CD00023074ADBB204785C4090
:100D8000135D401C491E0C06F7D1D843C0B210BDFC
:100D9000FF20C0B210BDC046927D00087047000021
:100DA00080B504480021818101604160816004F0C8
:100DB000ADFB80BD7401002010B5B6200F490C5A60
:100DC0000F4804800F480068FFF7F0FB0E49FFF75B
:100DD0001DFA0E4908602046FFF7F3FB0C49FFF7A8
:100DE00015FA0C4908600C480068FFF7DFFB0B4957
:100DF000FFF70CFA0A49086010BDC046C001002088
:100E00008C01002088010020F90215509401002077
:100E100000007A44980100209001002000401C4608
:100E20009C01002002480088024908827047C046A1
:100E3000AC0D00201C160020B0B5012004F030FDE0
:100E4000022004F02DFD074D6C7A002C09D0E868D3
:100E50002146FFF72BFCE86028692146FFF726FCB6
:100E60002861B0BD14110020F0B585B0421E91B2CA
:100E7000022900D9BCE10190DE4B18880090DE4FBA
:100E80003E8810B24000DD49095A3980DC4A1180A1
:100E9000DC49085ADC4908801880DC49088006F0E3
:100EA00078FD3A88DA4C2568B242029648D0052E81
:100EB00009D8D848D849C0467E4436797600B74428
:100EC000100205080B0EDD4800210AE0D948DA4976
:100ED00007E0D648D64904E0D248D34901E0CF48DC
:100EE000CF49D74B19605860052A08D8D149D24854
:100EF0007A44127952009744100205080B0ECF492C
:100F000000200AE0C349C44807E0D249D24804E0BF
:100F1000CE49CF4801E0CB49CB480CCBFFF766FA6E
:100F200006460F462846FFF753FB02460B4630465F
:100F30003946FFF75BFAFFF767FB0546AE4F029EA7
:100F4000C648056025602820052106F041FC206088
:100F50003A88C34C2568B24248D0052E09D8AD481E
:100F6000AD49C0467E4436797600B7441002050884
:100F70000B0EB24800210AE0AE48AF4907E0AB488B
:100F8000AB4904E0A748A84901E0A448A449AC4BF8
:100F900019605860052A08D8A649A7487A441279EA
:100FA00052009744100205080B0EA44900200AE0E5
:100FB0009849994807E0A749A74804E0A349A448ED
:100FC00001E0A049A0480CCBFFF710FA06460F46F7
:100FD0002846FFF7FDFA02460B4630463946FFF732
:100FE00005FAFFF711FB0546834F029E9B480560FB
:100FF0002560F820052106F0EBFB2060012041026E
:1010000098480491405A002871D00024964D0AE077
:101010000F4601C5E0B204F067FC92480499405ABB
:10102000641C844263D239463F882868B742EFD0B7
:10103000052E03901ED8B10002A253587649754A76
:101040007F4E9F46811000085D1000086310000865
:10105000691000086F1000087D1000080021774A11
:101060000EE07549734A0BE07149704A08E06E4919
:101070006C4A05E00021714A714E01E06849674AF7
:1010800006C6083E052F11D8B80002A10A586A48C2
:1010900068499746C9100008AD100008B310000851
:1010A000B9100008BF100008C510000800206349EF
:1010B0000AE05948574907E06748664904E0644830
:1010C000624901E060485F490CCEFFF78FF90646A0
:1010D0000F460398FFF77CFA02460B463046394626
:1010E000FFF784F9FFF790FA434F029E91E74148DA
:1010F00000880099814271D04B1E032B08D85B49B0
:101100005B4AC0467B441B795B009F44090104078E
:101110004A49002204E05949594A01E05549564AD2
:10112000474B1A605960401E0025032808D8554EC9
:101130002F46C046784400794000874409010407DF
:101140003E4E2F4604E0524E524F01E04E4E4F4F5E
:1011500003F0CEFC03F072FC4F4C03CC083CFFF7CD
:1011600045FA02460B4638463146FFF73FF902463C
:101170000B46334903C9FFF739F9FFF763FA07460E
:101180000E46464A2B46FEF7B3FF454A1060EB4336
:10119000444AFEF7DDFFC0192060434A10607141E8
:1011A0006160424E711D092201273B4600F084F820
:1011B0003B480068052231463B4600F07DF804F0CC
:1011C000FBF803F055FC00F0AFFB681C042D05464E
:1011D000F9D3374800210180364801605A48019907
:1011E00001801A20022106F017FBC0211D4A50522F
:1011F00005B0F0BDB20000209C100020867D0008E4
:101200009E1000208C7D0008B4000020B00000205B
:10121000E810002051B8AE3FB81E85EB5F34DE3FCA
:101220001188B2CA9AA92B40BD9AA9BB19513C405A
:10123000905F07CEAAAA3040ABAAAAAA0000F03F4E
:10124000D010002079F30040A8FCE02F4082B23F8C
:101250006D3480B7C514A23FE67367886011002023
:10126000F0100020C0010020C80F00204D62503F48
:10127000FCA9F1D2578EEA3F1A578E1A14FF9C3FF1
:1012800058A1B54700408F40AE47F33F48E17A147C
:1012900048A841402F0735E7A810002000CA9A3B14
:1012A00080110020003665C48411002074010020E4
:1012B0008A100020CC100020F0B581B014460D46F5
:1012C00006460027002B03D0F943002C03D115E07C
:1012D0000121002C12D0002B01D06019451E009175
:1012E0000A213046FFF7E2F9F621414389192970B6
:1012F00000996D187F1CA7420646F1D301B0F0BDDE
:10130000B0B51048018900290DD0F34A521E0023C0
:10131000C488651CC580515C05692955521E5B1C3B
:1013200001898B42F4D382888B1C934202D900211D
:101330008180B0BD4B080381511A81800188C91892
:101340000180B0BDA40100206811002080B50020FC
:1013500001F0CCFA042804D1A2480068002809D181
:1013600009E0002001F0C2FA022804D19D4840683B
:10137000002800D08047002001F0DCF980BDC04685
:1013800080B5012001F0B2FA042804D195488068A4
:10139000002809D109E0012001F0A8FA022804D1AF
:1013A0009048C068002800D08047012001F0C2F9B1
:1013B00080BDC04680B5022001F098FA042804D10F
:1013C00088480069002809D109E0022001F08EFA5E
:1013D000022804D183484069002800D080470320B8
:1013E00001F084FA042804D17E488069002809D1DC
:1013F00009E0032001F07AFA022804D17948C06993
:10140000002800D08047022001F094F9032001F069
:1014100091F980BD10B5694C2078FD210140217003
:10142000644801F001FB2078FE210140217000207A
:10143000152100F013F8A01C3E4C206120784001DB
:101440000549421821460C31204601F079F9204621
:1014500001F0E0FA10BDC0460090024080B582B0B5
:1014600001AA11705070012000025080104601F056
:101470004DF902B080BD0000F0B59BB00190002492
:1014800015212046FFF7EAFF2A4F384601F0CCFA33
:10149000BC7001256802029038804848801C46498B
:1014A000254AF96038617A612448386203AE3846CB
:1014B00001F040FA002800D0FEE72C36204F032030
:1014C00078703C701F480168232048430199FFF75A
:1014D000EDF8401E80B2FFF711FC1B492846FFF7CC
:1014E0002FFC03A8847404820299F1807471B57092
:1014F00013901648129016491191164904910397BA
:10150000154A0592034620330693144B08930B911A
:10151000791C0A910C920D9010203071348011A822
:1015200001F008FA002800D0FEE7024801F072FA44
:101530001BB0F0BDBC000020010000010101000152
:101540000C01002010000020310D000820010020B7
:101550000104000208A50240010001001000000281
:1015600010B5002414212046FFF778FF114884703D
:1015700001210A0202804A0242840F4A8182034604
:101580000C335975812149000C4B5918C160026117
:101590000B49595CC18201F0CDF9002800D0FEE76B
:1015A000044C02210122204601F0B4F9204601F04A
:1015B00031FA10BDE400002000380140B20D0020D7
:1015C0000302000010B5C300064CE150E1184A6068
:1015D000032805D840B2800003A1085806490860D6
:1015E00010BDC046481000200002000000040000AA
:1015F000000800000008000000E100E0F0B583B042
:1016000031480468314E7D200190C7007760600842
:101610000290F0603461642520462946FFF746F8C1
:1016200030600A2060432946FFF740F80546B06065
:101630002748844202D80198800030603068B84260
:1016400005D3052060436421FFF730F870607068AF
:101650008542029A02D880184008B060B068824281
:1016600002D800194008F06001204402194D0520FD
:101670002853194A10700221204606F0CDF8285B45
:1016800000281FD02A463D4600200646F1B21746E4
:101690004A00124B9D5289000C4A51580E4A116063
:1016A000D84B1D80598051889980072148432018C4
:1016B000001D80B206F08CF83A46395B761CF0B219
:1016C0008142E3D803B0F0BDE8100020C80F00202D
:1016D0004FC30000C0010020681100201810002036
:1016E00010B5054C0521204600F065F820210122A7
:1016F000204601F0DEFA10BD4008014080B501200F
:1017000001F09CF9012807D1012001F093F9244848
:101710000068002800D08047022001F08FF90128DE
:1017200007D1022001F086F91D484068002800D04A
:10173000804780BD80B5042001F080F9012807D1E1
:10174000042001F077F916488068002800D080470F
:10175000082001F073F9012807D1082001F06AF987
:101760000F48C068002800D0804780BD70B50C4D80
:101770001035042603E02D1D761C082E0FD0012005
:10178000B04084B2204601F059F90128F3D1204637
:1017900001F050F928680028EDD08047EBE770BDD4
:1017A0006810002001228A404168914341604169EC
:1017B00011434161704701228A40436813434360EB
:1017C000436993434361490003238B40016A994372
:1017D0000162016A01620169914301617047000081
:1017E00080B50648002101800120000303F062FF5C
:1017F0000348044906F0D4F880BDC04642110020D9
:10180000000C0040393200080648002101600648FB
:101810004178FE220A404270017825220A40803237
:1018200002707047C8030020BC0F0020F0B581B0E3
:101830000C46074680010C494618B8061B4D04D1DA
:10184000304631462A4601F001F9FF200230874236
:1018500002D3DB48042101761022304621462B4674
:1018600001F04AF901B0F0BD00400108F0B581B0C7
:101870000C46074680010C494618B8060B4D04D1AA
:10188000304631462A4601F0E1F8FF200230874217
:1018900002D3CB48042101761022304621462B4644
:1018A00001F02AF901B0F0BD00900108FFFFFF0030
:1018B000F0B585B00E27474301263002381803AC37
:1018C000072521462A4602F05DFF092080013818CD
:1018D00001A92A4602F056FFA57906212046FFF706
:1018E00047FA014600208D421BD101A9897903AA3C
:1018F00092798A4215D10020014603AA525C01ABBD
:101900005B5C9A420DD10F231A4003AB5A54092A4B
:1019100007D803AA002353544A1C05291146ECD3C7
:10192000304605B0F0BD0000F0B585B0324A107801
:10193000401CC1B2042900D90020107001210A0204
:1019400001922E4C04E01070029A511C032A4FD8C9
:101950000291C0B20E27474301983D18072628463A
:101960002146324605F032FF03A92846324602F0EE
:1019700009FF0020215C03AA125C8A421AD1401C94
:101980000728F7D1092080013D180726284621465F
:10199000324605F01BFF03A92846324602F0F2FE4C
:1019A0000020215C03AA125C8A4203D1401C072854
:1019B000F7D107E0104A1078401CC1B20429C2D9FF
:1019C0000020C0E70E480068A74C20600A48057850
:1019D00004212046FFF7CCF92071052255430198D8
:1019E0004019D030214605F0F1FE002005B0F0BDD1
:1019F000012005B0F0BDC046C4030020E40C002067
:101A0000CC10002060110020B0B5384C208803288D
:101A10001CD8C0467844007940008744011C334AF2
:101A200033480421817139498180012529050160EC
:101A300030480178FE220A40027003F0F1FDFF20D9
:101A400048302F490A881018088041E00020208083
:101A500003F02EFFB0BDFFF7EFF925480421817197
:101A60002849818028490160C16802694161C261D9
:101A700003F0D6FDFF20483021490A88101808805D
:101A8000022525E0FFF7D8F91948042181711A4988
:101A900081801A490160C16802698161026203F0B4
:101AA000BFFDFF20483016490A881018088003251A
:101AB0000EE0FFF7C1F90E48C16802694162826217
:101AC0000C48017801220A43027003F0F1FE04255C
:101AD00025800F4801680A480288914201D9491DB2
:101AE0000180008803F02CF8B0BDC046041100202E
:101AF00014110020A00100200711000000041000B4
:101B00000611002003110000000110000211000066
:101B1000242C014070B52A4902220A818A88012AB0
:101B200006D82848002202808A800320087670BDEB
:101B300000220A76234A01231380CA88531CCB80D3
:101B40000C69A55CCE4E7570921CCA8099B2615C1E
:101B500031703188018070BDF0B583B00446184DF6
:101B60000320287617480026068002272F81AF8899
:101B7000012F02D8AE8003B0F0BD019102922E7603
:101B8000EE88771CEF802869825DBD494A70B21CDF
:101B9000EA80BAB2805C08700D889D420DD8089822
:101BA00085420AD32088854207D001200549088054
:101BB0000198029905F030FE208003B0F0BDC046C8
:101BC000A4010020FE100020F0B583B00120C20364
:101BD00089200324214602F0EDFDC221CA4D68523E
:101BE0007D20C2008C20214602F0E4FDC421685211
:101BF000052001900002022100220090029202F0D2
:101C0000D9FD16490880000426D0154D154E029CBA
:101C100007E02880B61CAD1C641C10480088844274
:101C20001AD2019A1046604300990818801C80B2AD
:101C3000022360490F4602F079FD38463F790421BE
:101C4000FFF796F887420298E3D1002059490871BE
:101C5000488830800888DCE703B0F0BDC00F002062
:101C6000680000202000002060110020F0B58BB03B
:101C7000034602B20020002A00D589E0002900D0E6
:101C800086E04448834200D30346434883420AD354
:101C90004748484C0322214602F090FA0020E070A9
:101CA00020680BB0F0BD3D4801935843810C0320E0
:101CB00000914843C01E08AD0C22294602F07EFA6E
:101CC0000027FE43364806603648076004ACD94B0F
:101CD0003A4602973946039704E0241DED1C521C36
:101CE000042A17D00398D87028781870687858702C
:101CF000A878987018682060B84203D9294908600C
:101D000091B20746B042E8D2254E306096B20296B4
:101D10000646E2E700231846029D02E0531C032A10
:101D200009D21A468B42F9D0AA42F7D083B208AC46
:101D3000E254401CF2E708A801788A0004AB9D58E1
:101D4000194C25604778B8001858421B174E32606E
:101D5000062318464843791A594389B20523DB43C1
:101D6000009F7B43019FFB189B1D9BB2984206D2AC
:101D7000181A5043FEF79AFC3060401905E0C01A6B
:101D80005043FEF793FC3060281A2060C117884347
:101D90000BB0F0BDF47F0000DD7F0000ABAA0000B7
:101DA0008411002080110020881100208C11002057
:101DB000F63F00006011002080B5002000F090FD8B
:101DC0000249401A801E024A885480BDB20D00208C
:101DD00002020000F0B581B09C4EF089274988428C
:101DE00001D2254843E0B08C924F388080200324F4
:101DF000214605F011FD23490880F08A38807720BC
:101E0000214605F009FD20490880B08E3880ED207C
:101E100085002846214605F0FFFC1C4908803089D2
:101E2000388009352846214605F0F6FC1849088017
:101E3000F08C38809520214605F0EEFC154908808D
:101E4000708C38809B20214605F0E6FC1249088002
:101E5000B0893880AA20214605F0DEFC0F490880B1
:101E600003F0B6FC0920C0027949097808187849BE
:101E7000088001B0F0BDC046524500009F39000007
:101E800068110020CC030020F60C0020B8000020D0
:101E9000F00C0020D80C0020DC0C0020D40C00201A
:101EA000C01C062803D8800003A1085870470148C9
:101EB0007047C04640420F00010000000A000000C9
:101EC00064000000E803000010270000A086010065
:101ED00040420F0070B50D204001D54908180B4C49
:101EE000206000250A4E725D0321084668430B02FC
:101EF000C01880B202F05EFC21680880881E206055
:101F00006D1C302DEFD170BDC0010020600100209C
:101F1000927E0008F0B581B0BC4D2888FF260146AE
:101F2000B143424A8918090A05290AD8794409792E
:101F300049008F44020620244F5302F071F901B08A
:101F4000F0BD0F21090301400722520391426AD1DB
:101F5000C2490988AE4A914265D1C2494018E98810
:101F60002A695118AA88B14B1B88002B59D002F05E
:101F7000F1F801B0F0BD02F0EFF901B0F0BDA888B2
:101F8000022850D32D4CAB4F2D4E0AE01030C00626
:101F9000800EAF49085A3880FFF7B2F9A8880128A7
:101FA00041D90220288128880F2201469143A1426D
:101FB000ECD0B142EAD083221202914205D1400016
:101FC000204940182049405AE1E7800A20282AD8B1
:101FD0000020E0E702F048FB01B0F0BDA88802282D
:101FE00021D3134F934C06E000202080FFF788F99F
:101FF000A888012817D90220288128880146B143E2
:102000003A46203A92B29142EED1B8420BD8400003
:102010000949401880B202222146134602F086FB8D
:10202000E4E702F08BF801B0F0BDC0460080FFFF8E
:10203000208500006811002000FCFFFF20830000C5
:1020400010830000CE7E000800FAFEFF1C16002060
:10205000AE0D0020F0B581B06C4F0020388101F04A
:102060007DFA002801D001B0F0BD6B4D704C08E046
:102070002046BC30022105F041FC01F06FFA002837
:10208000F1D1022038813E88AE420BDD63498E4299
:102090001DD063498E42EBD062498E4209D10221A4
:1020A0006248E8E70121C9038E4230D05E498E4282
:1020B000E3D0310B0E2900D0A4E0684800885449D1
:1020C000884278D00420387605F063FCD5E72C46AA
:1020D000F9884A1CFA803B695E5C564D6E70891C1B
:1020E000F98091B2595C29702988534A914228DDC0
:1020F000484A914233DC53488142254648D04548FE
:1021000081424B4C54D1434854490880B5E70226DC
:102110002046314605F0F2FBA01C314605F0EEFBEF
:10212000201D314605F0EAFBA01D314605F0E6FB17
:1021300020460830314605F0E1FB20460A303146A2
:1021400099E74148814227D03148814225462BD02A
:102150003E488142364C2BD1FFF73CFE8DE7374A93
:10216000914225461ED0364A9142314C20D1384901
:102170008989BC22A152374A10702E480180364806
:102180000078552800D178E7AA203349087074E711
:1021900001F056F8264C70E730482B49018025465F
:1021A000234C6AE71B48401C2C490880204C64E7FC
:1021B0000420387661E7F88839690918BA88284810
:1021C000FDF7DEFF0120400330181849098880B26E
:1021D000002903D02249FFF749FB02E02049FFF71D
:1021E00025FB38881F494018BA881F4C214601F04A
:1021F000B1FFBA881A482146FDF7FBFF002800D13D
:1022000031E70420387601B0F0BDC046A4010020BB
:1022100054430000314E00000182000002820000A1
:10222000168200001782000006800000F6100020D1
:10223000C001002068110020534C0000324E000005
:1022400057500000544C0000544100005448000016
:102250001C160020F5100020F4100020AE0D002008
:102260009C1500200020FFFFDC1500200146002007
:10227000632904DC012901D00A2906D170476429A9
:10228000FCD07D22D2009142F8D00120704700009E
:10229000F0B583B001AC0025A57181204000A0807D
:1022A00002200190504E3046214600F077FCA57187
:1022B00001273802A0800C4801903046214600F0EA
:1022C0006DFC304639462A4600F0F3FCA571FF202C
:1022D0000230A080474805700197403E30462146B5
:1022E00000F05CFC03B0F0BD01000100F0B581B06E
:1022F0003D4C0221204600F0D5FC05463B480178C4
:102300008D4206D13A480188491C8AB28A4203D0DC
:1023100003E0057036480021018035480088022816
:1023200060D3344F3878012817D13348007801281A
:1023300013D12046403820210026324600F0B9FC57
:1023400001212046324600F0B4FC642005F00FFB6A
:102350002A4806603E7028480670387801281CD04C
:1023600000283FD1012D38D125480078002839D1E7
:10237000224E3068401C3060322833D3012520467D
:1023800029462A4600F095FC642005F0F0FA00206A
:1023900030603D701849087022E0012D1DD11848A9
:1023A000007800281ED115490868401C08603228B2
:1023B00018D32046403820210026324600F079FC10
:1023C000012520462946324600F073FC642005F0C2
:1023D000CEFA0A4806603E7002E008480025056013
:1023E0000748057001B0F0BD40080140B61000205C
:1023F000B4100020B2100020B0100020B81000204F
:10240000B71000200249012800D02C31086870471D
:102410009C280140054A012800D02C32106802296E
:1024200001D0012070478007C00F704798280140F5
:102430000B4B012A05D101280AD1186808431860FE
:102440007047C943012807D11868084018607047D1
:10245000D86A0843D8627047D86A0840D862704783
:10246000A028014070B50C460646012528042946DF
:1024700001F002FE002C62D0022E2DD0012E5ED182
:102480000121480201F0F8FD3048C169304A0A4094
:10249000C26121788900C2690A436178C902114387
:1024A000C161E178A27852010A430262A1798902EE
:1024B000227A52020A43617A09021143E279120137
:1024C0000A432179114341626179816201680222E4
:1024D0000A430260002070BD0125A802294601F0D0
:1024E000CBFD1A48816C1A4A0A408264217889001F
:1024F000826C0A436178C90211438164E178A27851
:1025000052010A43C264A1798902227A52020A4323
:10251000617A09021143E27912010A4321791143D8
:10252000016561794165016804220A43026081689E
:10253000A27A012A05D1AA04114381600025284608
:1025400070BDAA0491438160002070BD88280140BD
:10255000C3C7FFFF401E4142414188020121890259
:102560000F4A13688B4318181060704701214A0303
:102570000B49012803D10868104308607047C86AF6
:102580001043C8627047C0460549064A012803D176
:102590000868104008607047C86A1040C8627047F9
:1025A000A4280140FFDFFFFF70B50D460446012659
:1025B0007002314601F044FD2878401E411E8841DA
:1025C000400021680222914308182060A878401E2C
:1025D000411E88412168B143081820606878401E78
:1025E0004142414188002321C900625804239A4393
:1025F0001018605070BD00000849002804D0012860
:1026000007D0022804D070470868012202430A60FC
:1026100010310868012202430A6070470CA502408D
:1026200000280FD002281FD0012836D136480129B2
:1026300026D1416801220A434260016802220A430E
:1026400002607047304801291FD1416801221143BF
:102650004160416911434161016802229143016077
:1026600001691143016170472748012916D1416969
:1026700001220A434261016902220A430261704752
:10268000016802229143016070470221C943026838
:102690000A40026002690A40026170470169022231
:1026A000914301617047C046002806D0022808D037
:1026B000012805D1044801607047034801600161A9
:1026C000704701480161704700A5024000280FD003
:1026D000022807D0012816D10B4801680122914336
:1026E0000160704708480169012291430161704708
:1026F0000120C24304480168114001600169914210
:1027000000D3891C0161704708A5024010B504463A
:102710000120014601F094FCE078C001A178890114
:102720000143207808436178014A8854002010BD95
:1027300000A00240014908707047C0461F80024057
:10274000F0B583B0044608681060486810618F7D5A
:102750003802C019D08001252B46BB40487D102887
:102760000190029505D1088B58439080488B4343D4
:1027700000E0938093820B890420165E1420155E7E
:10278000C87D052845D80094029C2404BC4024142C
:102790005C43E7177C40E71B5E435D437844007968
:1027A00040008744020B1A2902024A4807409760FA
:1027B000488946437342D360454327E04448074075
:1027C000704203039B08FB18029CE4071B199360EB
:1027D000D06048896843454219E03D4807406D4252
:1027E000280380083818029B9B07C018906048890E
:1027F00070434042D0600AE035480740B002381AC2
:1028000003239B07034393607042D0606D42956140
:10281000009C4889D083D08200209083607804286F
:1028200029D002280DD001284FD10198C007000FF0
:102830009083D08B28490840D083D08A0840D0822A
:1028400043E0087D0102019BDB071B0F5918203173
:102850009183D18B204B1940D1834002D18B01430E
:102860001E4C2143D183D18A1940D182D18A0143A0
:102870002143D18229E0487C8000019BDB071B0FAC
:102880000343087C400018438B7C0343102018430B
:102890009083C8689061D08B0F4B1840D083D08A4A
:1028A0001840D082087D10280FD0D18B43021943E5
:1028B0000A4C2143D183D18A19432143D18200029A
:1028C000918B0143202008439083002003B0F0BD8A
:1028D000FF030000FF3F0000FF7900000080FFFFC2
:1028E000400101494058704710900240400148495A
:1028F0004018818B490709D5C18A054A0A40C08B17
:102900004008C0B2824201D80420704702207047BC
:10291000FF01000010B500784001054BC45A012AA0
:1029200002D00C40C45210BD0C43C45210BDC0466E
:102930001C900240F0B581B0054601242046214696
:1029400001F07EFB31490868002846D42878887653
:10295000C877887780220A60697804293FD1A868FF
:1029600000284BD06868002848D00094E8780028F8
:1029700015D000273C463E46A868C1194889002862
:102980003FD0088900283ED0686802192846FFF722
:10299000D7FE1C372034761CE8788642ECD3686872
:1029A00001682A7852011A4BD150D11882888A8046
:1029B000C288CA8082688A60C268CA6002690A6185
:1029C000828A8A82C28ACA8282698A6100248C834E
:1029D000828B8A83C08BC88310E002240EE0E98AD0
:1029E00000290BD0A98A002908D029460C314001C2
:1029F000074A82182846FFF7A3FE0024204601B0AC
:102A0000F0BD009CFAE7009CF8E7C0460080024059
:102A1000009002400178034A11708078012800D1AB
:102A2000917070471B800240007801490870704720
:102A30001A800240044908607047C046024909688C
:102A40000840411E8841704714040140F0B581B030
:102A50000123884244D8244CA14241D8234C134638
:102A600025460C3D2F6830263E4003D05F1E002BCC
:102A70003B46F5D1002E01D0022331E0EFF3108365
:102A80000093EFF3108372B6884206D9184820608D
:102A9000009880F31088002322E00023DF43154BC9
:102AA00023602346143B18602646183E01233360FA
:102AB0007A431E038019BFF34F8FBFF36F8F2E68C9
:102AC000760603D4521C012AF9D104E07A438842E5
:102AD000084BE5D9DAE706482060009880F31088B3
:102AE000184601B0F0BDC04600D001081C3C0040B3
:102AF000DCFE658723019A78F0B582B0C50E01240B
:102B0000002D43D0234D4619361DAE423ED3224DF3
:102B10001C462F6930263E4003D0671E002C3C46E1
:102B2000F7D1002E01D0022430E00191EFF310869E
:102B3000EFF3108472B62F68012427432F60002A18
:102B40001DD00027F9430091019980C9019180C0EF
:102B500000994B43BFF34F8FBFF36F8F521E2F6906
:102B60003F0608D42F68A7432F6086F310885B1CAC
:102B7000012BF4D10AE000994B431704E4D12868F3
:102B800001218843286086F310880024204602B083
:102B9000F0BDC0460020FEF7003C0040F0B583B019
:102BA0000C46054680200121029101F049FA268851
:102BB000002E75D000210A460B46019617E0A86842
:102BC000B843A860E868B843E8600F2090402E68DA
:102BD00086432E60A07990402E6806432E60019EA9
:102BE0005B1C3046D840891C121D002858D0029F1B
:102BF0009F403742F4D0A678022E16D0012E08D07E
:102C0000002E23D16E68BE436E606E693E436E61D6
:102C10002BE06E683E436E602E69BE432E61032634
:102C20008E40286AB04328620AE0686838436860CA
:102C3000286938432861032088402E6A86432E6223
:102C4000E07888402E6A06432E620EE06868B8433A
:102C500068606869B8436861A869B843A861A868F2
:102C6000B843A860E868B843E8606079002802D0FB
:102C7000A869384301E0A869B843A8612679022E03
:102C800008D0012E9BD1E868B843E860A8683843B3
:102C9000A8609AE7A868B843A860E868384393E753
:102CA00003B0F0BD406A0840411E8841704741634F
:102CB0007047002A02D02C22815070473022815068
:102CC0007047000070B50022002934D0814232D212
:102CD000420802439008104302090243100A1043BD
:102CE000020C0243D0434308144A1340C31A144849
:102CF0009C08034004401B191C091D19114B1D4061
:102D0000114C65432D0E4E080E43B10831430E0998
:102D10000E43310A31430E0C0E43F1434E08164068
:102D2000891B8A0801400240881801094018184090
:102D30006043000E421BD0B270BDC046555555557C
:102D4000333333330F0F0F0F01010101044948687A
:102D5000C00702D100200860704701207047C046BC
:102D600010300040016880220A4302607047000072
:102D700080B50021016041608160C1600161012274
:102D8000254B984203D0D00701F068F980BD900729
:102D900001F064F980BDC0460268802313430360DC
:102DA000491E4A424A419101026840239A43511800
:102DB0000160704770B50D460446012616488442EE
:102DC00001D0F00700E0B007314601F047F9206874
:102DD000B04320602878411E8841400021680222CB
:102DE000914308182060E878411E884180002168DE
:102DF000042291430818206060687F218843606046
:102E0000A878810811406A78636813430007400E70
:102E100018430843606070BD000C00408160016889
:102E200081220A4302607047F0B583B00E46044623
:102E30000125A803324F39688143226812030240FA
:102E40005018386000BF2078C0070AD001A90220BE
:102E50008871002088700D80280288801948FFF74B
:102E60009DFE2068032108403A688A4311183960A2
:102E700000BF711C3A681207920F904202D0491E9F
:102E8000F8D11CE000BF3868F0218843616809016F
:102E90000143396000BF072001023A688A43A168F4
:102EA00009021143396000BFC00239688143E068FC
:102EB000C0020843386000BF02F054FD00252846D8
:102EC00003B0F0BD400801400D4800684005400FC8
:102ED000042801D3C11E00E000210A480068C84050
:102EE0007047C046064800688004400F042801D39C
:102EF000C11E00E0002103480068C8407047C0467A
:102F0000041002401000002070B50546012420077F
:102F10000F4E316801433160E00631680143316092
:102F2000204601F037F87068012D09D12043706008
:102F300008487168890708D4401CFAD3204670BD40
:102F4000A04370600024204670BD002070BDC046C4
:102F50001C1002400000FFFFB0B504460125280404
:102F6000294601F089F8002C28D0154801682278FC
:102F7000042A02D1082291430AE0FF230433994333
:102F8000016001680A4361780B0213430821194369
:102F90000160A2780168042A02D1402291430BE02B
:102FA00023231B0199430160110102680A43E17860
:102FB0004B02134340211943016000252846B0BD50
:102FC0001C280140F0B581B001223349314B1C4629
:102FD00002E0641C012E07D0664266410F8820255E
:102FE0003D40F6D01646F4E70124002D17D002E04C
:102FF0005B1C012E07D05E425E410F8808253D40D4
:10300000F6D01646F4E7002D09D00A8882430A80DC
:103010000024800703D501204002FFF70BFD204666
:1030200001B0F0BD10B51B4A1B490C880823234092
:1030300003D1541C002A2246F7D1002B01D10120D4
:1030400010BD8A8A098B120451180160002010BD3E
:10305000114909880840411E8841704710B50D4A42
:103060000D490C882023234003D1541C002A2246FA
:10307000F7D1002B01D1012010BD0A8810231A437B
:103080000A80020C8A8308840888984308800020FC
:1030900010BDC0460100FFFF04280040574A4A40C7
:1030A00002617047002A03D0C2680A43C2607047B9
:1030B000524A5140C2680A40C2607047B0B50D46DE
:1030C00004461348844204D00120014600F0C6FFA4
:1030D00003E00121C80200F0CFFF20686988E162A7
:1030E0002988A16269794A1E9141C9013F221201D2
:1030F00090432A790243E888104380229043401885
:103100002060606901210143616100202061B0BD40
:10311000002C0140016801220A4302607047000050
:103120000168024A0A4002607047C046FEFF000084
:1031300002460020022909D004290ED15168C9078E
:103140000BD05169C90708D0012070475168890721
:1031500003D55169890600D501207047F0B581B0CB
:103160000D46044624480121844205D0480400F05D
:1031700075FFFFF7A9FE04E0880300F07DFFFFF76D
:10318000B1FE070900952D6838462946FDF78EFAED
:10319000064628467043381A000169084018294637
:1031A000FDF784FA0F2800D9761CE049E26FD207B8
:1031B00006D04A1E09041146F8D1032001B0F0BD23
:1031C000E26880210A43E260F2B22260320AD2B29F
:1031D00062600F221040C022A050009B9888DA88BD
:1031E000024318891043E2680243E260E0688843C2
:1031F000E060002001B0F0BD00380140FFFF00009A
:1032000080B504480068002800D080470248FFF7D6
:10321000A9FD80BDDC100020000C004080B50448F2
:103220000068002800D080470248FFF79BFD80BD62
:10323000E0100020200C004080B502F081FA80BD33
:10324000F0B581B0264EF0892749884201D925483A
:1032500041E0B08CB44F388086200324214604F02E
:10326000DBFA22490880F08A38807D20214604F06C
:10327000D3FA1F490880B08E38801E4D284621465B
:1032800004F0CAFA1C49088030893880093528467C
:10329000214604F0C1FA19490880F08C3880922048
:1032A000214604F0B9FA16490880708C38809820BD
:1032B000214604F0B1FA13490880B0893880A7206C
:1032C000214604F0A9FA1049088002F081FA0F485B
:1032D000407800024C300D49088001B0F0BDC04676
:1032E0001C16002052450000A5270000CE03002038
:1032F000F80C0020B1030000BA000020F20C0020FE
:10330000DA0C0020DE0C0020D60C0020AE0D0020D0
:10331000F0B581B09A4C0025257620694178C91E08
:10332000402900D941E0C0467944097949008F44D9
:10333000203C3C3E3C4F3C3C3C3C3C3C3C553C3CBB
:103340003C3C3C3C3C3C3C3C3C3C3C3C3C3C3C3CBD
:103350003C3C3C3C3C3C3C3C523C3C3C3C3C3C3C97
:103360003C3C3C3C3C3C3C3C3C3C3C3C3C3C3C6574
:103370006800C1788278120251182180427903795D
:103380001B029A18A28093B2332B34D209B2520096
:103390006281A28082700320E0806089001D6081CC
:1033A000002940D403F0E8FA3FE0012024E0C1788E
:1033B000807807226281404A6260000240182080C3
:1033C000411C618000B200282AD403F0E5FB2CE008
:1033D0000078002829D1FDF737FB26E0C1788278F4
:1033E000120251182180427903791B029A18A28097
:1033F00093B2332B08D30420207616E0FDF7F0FAC1
:1034000013E0FDF79FFB10E05300A380511861808B
:10341000102141700720E0806081605F0028D4D5D2
:10342000FEF718FE01E0FEF775FD207E00280BD0A8
:1034300021694A78802313434B70216901228A70E5
:103440002169C870052060812069017800292ED08B
:103450006189002929D00A46FE32D2B2334F344B5B
:1034600004E06E1C9542274635460BD0445D7C40F7
:10347000082702E034467F1EF3D06608E407F9D03F
:103480005E40F7E7284A1480537843543C4B186950
:1034900059890818401E117801705889421C5A81B8
:1034A0005869196992B2FCF76BFE01B0F0BD0020BB
:1034B000608101B0F0BDC04602000400F0B53049A3
:1034C000002048818A89052A2AD3A223154C012588
:1034D000E55209690B78012B22D15018431E1B7845
:1034E000114C6370801E00782070FD32D2B22088AB
:1034F00000240E4E0E4B04E0671C94422E463C46C0
:103500000BD00D5D7540082602E03D46761EF3D0D7
:103510006F08ED07F9D05F40F7E7411B484248418B
:10352000F0BDC046C001002068110020FFFF000070
:1035300001A00000124881880289931C8B4203D9A4
:10354000002181800120704753080381891A8180FE
:103550000188C918018000207047C04608490A89BF
:103560008B88012093420AD39B1A8B809BB2022B3B
:1035700005D3500808810A88101808800020704779
:10358000A401002080B50D480168491C01600A298A
:1035900005D3002101600A482021FFF788FB094874
:1035A0000168491C01600848814202D30748012193
:1035B0000170FEF79BFE03F02BF880BDD8100020B1
:1035C000000801404C11002041190100B0100020FA
:1035D00010B50020A04980220B4600241C70521E0A
:1035E0000833002AF9D1491C401C0828F3D110BD2A
:1035F000F0B583B00292994222D20A460299091A82
:103600000191C400944D29190091114604E0521C07
:10361000491CCCB29C4213D2029CA042F7D2D408DF
:10362000009D2F1907240C400125A540EC43019D66
:103630003E7826403E706D1E0837002DF8D1E6E733
:1036400003B0F0BDF0B583B00292994222D20A468F
:103650000299091A0191C400EA4D291900911146F5
:1036600004E0521C491CCCB29C4213D2029CA042E2
:10367000F7D2D408009D2F1907240C400125A5403E
:10368000EC43019D3E7826403E706D1E0837002DAC
:10369000F8D1E6E703B0F0BDF0B583B002929942ED
:1036A00021D20A460299091A0191C400D54D29195F
:1036B0000091114604E0521C491CCCB29C4212D22B
:1036C000029CA042F7D2D408009D2F1907250D4077
:1036D0000124AC40019D3E7826433E706D1E0837A4
:1036E000002DF8D1E7E703B0F0BDC046F0B583B0D8
:1036F00001AD0024AC71012000900702AF80524858
:103700000190524E30462946FFF748FAAC71AF801F
:103710004F480190304640302946FFF73FFAAC71E0
:10372000AF804C48019030462946FFF737FA4025D4
:10373000304629462246FFF7BCFAC827384604F02F
:1037400016F930462946009AFFF7B3FAAE20214613
:1037500000F052FB0220214600F04EFB10202146D3
:1037600000F04AFB2846214600F046FBB0202146E7
:1037700000F042FB8120214600F03EFBCF20214695
:1037800000F03AFBA120214600F036FBA62021469E
:1037900000F032FBA820214600F02EFB3F202146FE
:1037A00000F02AFBAD20214600F026FB8B202146AD
:1037B00000F022FB3320214600F01EFB3846214654
:1037C00000F01AFBD320214600F016FB20462146CC
:1037D00000F012FBD520214600F00EFB802630467B
:1037E000214600F009FBD920214600F005FB1F20EF
:1037F000214600F001FBDA20214600F0FDFA1220FC
:10380000214600F0F9FADB20214600F0F5FA2846BF
:10381000214600F0F1FAFC480146324600230B70C5
:103820000831521EFAD1401C641C082CF4D1092026
:10383000C101F448FCF7CBFC00F010F8AF200021E8
:1038400000F0DAFA03B0F0BD1000020140080140B8
:103850000100020140000101D4030020F0B585B051
:103860000020009002905038C0B2009D294600F020
:10387000C3FA0220294600F0BFFA10242046294648
:1038800000F0BAFAE14E403E049601273046214648
:103890003A46FFF70EFADD4839463A46FFF709FA8D
:1038A000304621462A46FFF704FAD84839462A46C8
:1038B000FFF7FFF978242E46E0B2C20910210498E0
:1038C000FFF7F7F90127D14D284639463A46FFF769
:1038D000F0F90022284639461546FFF7EAF9701C30
:1038E0006400072E0646E7D31021012704983A46C4
:1038F000FFF7DFF9C54C204639463A46FFF7D9F9BC
:10390000204639462A46FFF7D4F94024E0B2C209DE
:1039100010210498FFF7CDF90127BC4839463A46F3
:10392000FFF7C7F90026B94839463246FFF7C1F913
:10393000681C6400072D0546E8D310210124049873
:103940002246FFF7B6F9B14D284621462246FFF739
:10395000B0F9284621463246FFF7ABF930463546E6
:1039600001960390C000EF4908180299475CA74EE2
:10397000F8B2C20910210498FFF79BF901243046E0
:1039800021462246FFF795F9002230462146FFF7EF
:1039900090F9681C7F00072D0546E9D3102101240A
:1039A00004982246FFF785F9304621462246FFF764
:1039B00080F9002230462146FFF77BF90398401C2E
:1039C0008028019DCDD110240022049E304621463E
:1039D000FFF76FF901278D4839463A46FFF769F935
:1039E000304621463A46FFF764F90298401C082801
:1039F00000D037E70920C2018248CA49FCF7C0FB62
:103A000005B0F0BDD4030020F0B585B000237D4C97
:103A1000C44DD9006218125C6918095C914205D145
:103A20005B1C59B20029F4D505B0F0BD02905038A6
:103A3000C0B20027394600F0DFF90220394600F015
:103A4000DBF910263046394600F0D6F96F4D403D7F
:103A50000124284631462246FFF72BF96B482146C0
:103A60002246FFF726F90495284631463A46FFF7E5
:103A700020F9664821463A46FFF71BF97825634E40
:103A80000397E8B2C20910210498FFF712F9012741
:103A9000304639463A46FFF70CF90024304639469D
:103AA0002246FFF706F903994F1C6D000729E7D35B
:103AB0001021012704983A46FFF7FBF8534D28469A
:103AC00039463A46FFF7F5F8284639462246FFF7C9
:103AD000F0F840254D4EE8B2C20910210498FFF7D6
:103AE000E8F80127304639463A46FFF7E2F8002267
:103AF000304639461746FFF7DCF8601C6D00072C8E
:103B00000446E8D310210124049E30462246FFF7E4
:103B1000D0F83E4D284621462246FFF7CAF82846EF
:103B200021463A46FFF7C5F816E010210124304639
:103B300022463546FFF7BDF8344E30462146224630
:103B4000FFF7B7F8002230462146FFF7B2F8049F8E
:103B50007F1C802F2E4642D00497F9002948401838
:103B6000029A855C6F4B59188F5CAF4217D10027C2
:103B7000E9B2CA0910213046FFF79BF80124234817
:103B800021462246FFF795F8002220482146FFF7FC
:103B900090F8791C6D00072F0F46E9D3C5E7801810
:103BA0000390881801900025F9B2CA091021304607
:103BB000FFF77FF80124F64821462246FFF779F8FF
:103BC0000022F3482146FFF774F8691C7F00072D97
:103BD0000D46E9D301990978039A1170A5E71024DD
:103BE000002230462146FFF764F80127E8483946AD
:103BF0003A46FFF75EF8304621463A46FFF759F855
:103C000005B0F0BD54080020D40300208008014016
:103C1000F0B58AB006910590082B03D10624002C3C
:103C20000AD175E05907D808002900D0401C59086E
:103C30004143CCB2002C6BD00F98099058080290E9
:103C4000203AD0B2002501900001334908180090B5
:103C5000059A0493039404E00246089D6D1CA54256
:103C600056D0082B089504D10620019948432C49C9
:103C70000EE0182B08D0102B48D00C2B48D10C206C
:103C800001994843254903E02420019948432149EB
:103C9000081840190792D6B20478002306990DE05F
:103CA000099A002A16D0F2001E4DAA18D55D9D4330
:103CB000D555431C491C6408072811D2184607270C
:103CC0000F400123BB40CFB2FF08E207E8D0099ABA
:103CD000002AE8D0F200134DAA18D55D1D43E7E78E
:103CE0000798401C049B082B039CB5D0C1B2059AD1
:103CF000891A029A9142089D02D1069A08320692C8
:103D0000029A9142059AA9D00246A7E70098C0E717
:103D10000AB0F0BD908B0008A08500082C81000837
:103D2000047F0008D4030020F0B585B002AC07C4BE
:103D3000002B36D01C460A9D6808082D00D1801C37
:103D400001900B9F002610E0009730200143CAB27B
:103D50000198704302994018C0B203992B46FFF7AF
:103D600057FF761CF0B2A0421BD2F04300190106A7
:103D700006D001210A225143401E0206FAD100E07A
:103D800001210498FCF792FC0A21FCF78FFC002922
:103D9000DAD100970198704302994018C0B23022DE
:103DA000DBE705B0F0BDF0B583B0064617783846BE
:103DB0002038C0B25E281CD8082B01D05D0800E076
:103DC000062508980190541C029501980090F0B2C5
:103DD000FAB20D461F46FFF71BFF3B462946029DE0
:103DE0007619601C27783A46203AD2B25F2A0446F8
:103DF000EBD303B0F0BD0000F0B583B000910190AB
:103E0000634F3D46403D1024012628462146324658
:103E1000FEF74FFF384631463246FEF74AFF00278D
:103E20000295284621463A46FEF743FF5848314658
:103E30003A46FEF73EFF7824554EE0B2C209102103
:103E40000298FEF736FF0125304629462A46FEF73E
:103E500030FF002230462946FEF72BFF781C640015
:103E6000072F0746E9D31021012502982A46FEF7BD
:103E700020FF474C204629462A46FEF71AFF002716
:103E8000204629463A46FEF714FF0098002818D02D
:103E900040243F4EE0B2C20910210298FEF709FF0C
:103EA0000125304629462A46FEF703FF0022304608
:103EB0002946FEF7FEFE781C6400072F0746E9D36B
:103EC00016E00024324E1021002502982A46FEF703
:103ED000F0FE0127304639463A46FEF7EAFE304604
:103EE00039462A46FEF7E5FE601C072C0446EAD355
:103EF0001021012502982A46FEF7DBFE244C2046BD
:103F000029462A46FEF7D5FE0027204629463A468E
:103F1000FEF7CFFE019C1E4EE0B2C20910210298AE
:103F2000FEF7C7FE0125304629462A46FEF7C1FEA8
:103F3000002230462946FEF7BCFE781C6400072F9D
:103F40000746E9D3102101910127029C20463A46F9
:103F5000FEF7AFFE0E4E304639463A46FEF7A9FE52
:103F60000025304639462A46FEF7A3FE2046019C2E
:103F700021462A46FEF79DFE304639463A46FEF770
:103F800098FE029821463A46FEF793FE03B0F0BD34
:103F900080080140401E41424141080201210902BE
:103FA000024A13688B431818106070470070004075
:103FB000F0B581B06320E04C03260225214632464D
:103FC0002B4600F0B3FBA77820462946FCF7D0FE2D
:103FD000874201D0304600E02088C621D84F785271
:103FE000E620214632462B4600F0A0FBA67820466C
:103FF0002946FCF7BDFE864201D0E84300E0208858
:104000000D490880662021462A462B4600F08EFB8B
:10401000657801212046FCF7ABFE854201D00020E7
:1040200000E02078C0B2C821785204484178EF22DD
:104030000A40427001B0F0BDB00D0020A001002088
:10404000054A002903D011680143116070471168C7
:10405000814311607047C04614100240054A002990
:1040600003D01168014311607047116881431160EA
:104070007047C0461C100240054A002903D0116851
:104080000143116070471168814311607047C04659
:104090001810024080B582B00220FEF7D9FF012837
:1040A00009D10220FEF78EFF01A8FEF7BBFF0198A1
:1040B000001DFEF7D3FF02B080BD80B582B00120A5
:1040C000FEF7C6FF012805D10120FEF77BFF01A8FE
:1040D000FEF7A8FF02B080BDB0B500218F48084AA6
:1040E000C3885C1CC480545C30340569EC54491CA2
:1040F0000C29F5D10C210181FFF71CFAB0BDC04697
:1041000074010020B0B50C46054601F019F8A02056
:10411000204301F05DF8280A01F05AF8E8B201F0F6
:1041200057F801F00DF8A120204301F051F800F0FC
:10413000DBFF044601F02CF82046B0BD80B50B46ED
:104140005043034941181846FCF71AF880BDC04691
:104150000040010880B50B4650431C4941181846E1
:10416000FCF70EF880BDC0466F480C490180032063
:1041700040027149088010480188A0220A43028049
:104180007047C0466848054901806B480449018072
:104190000948018805220A43028070475443000001
:1041A0000680FFFF644840210180A52000020249EB
:1041B0000A8802430A807047C20F002080B50B4670
:1041C000024941181846FBF7DBFF80BD009001084B
:1041D000B0B50C46F94DE9882A695118AA8802231E
:1041E00000F0A4FA2C81E8880019E880FFF7A2F912
:1041F000B0BDC0460020704770B500290BD0EF4A13
:104200000B460478D5886E1CD680166974555B1EE3
:10421000401C002BF5D1E9480181FFF78BF970BDF7
:10422000F0B581B0E54CA088022800D274E03D4E84
:10423000E54F434D02E0A08801286DD9022020817E
:1042400021888A19092A17D87A441279520097448A
:1042500007090B0D0F110413133B00F04FFBEAE7A6
:10426000288840E068883EE0A8883CE0E8883AE09A
:10427000288938E0688936E000223A80284A91424D
:1042800032D30A0A802A47D8254A6C3292B2914228
:104290002AD8234A5218143A91B22A4B5943490C4E
:1042A000C04348438018EE4A1288204B9A421ED0E1
:1042B0001F4B9A4218D14900254A525A3A6080B29F
:1042C00002281BD1234825E0E54800881749884289
:1042D00005D01749884205D11848008803E01548E1
:1042E000008800E000203880FDF70AF8A3E74900C5
:1042F000154A525A3A6080B202280AD0012806D0E4
:104300000028F1D104202081FCF7FAFF93E7788898
:10431000E9E70E48405AE6E701B0F0BDA4010020ED
:104320000A8000000080FFFFAE0D0020324E00002A
:10433000314E0000C00F002068110020C40F002083
:10434000C0010020ABAA000020000020680000206F
:104350001A0D0020640D002070B5E94CA0880228D9
:1043600000D225E1964DF04E08E0E849085A308029
:10437000FCF7C6FFA088012800D819E1022020819F
:1043800020884119672900D972E049007944898859
:1043900049008F4469006D00730076006D006D0068
:1043A0006D006D006D006D0079007C007F00820063
:1043B0006D006D006D006700850088008A006D004B
:1043C0008E0090009300960098006D006D000E0125
:1043D0006D006D009B006D006D006D006D006D0047
:1043E0009E006D006D006D006D006D006D006D0034
:1043F000A100A300A600A800AB00AE00B100B4006D
:10440000B700BA006D006D006D00BD006D00C10009
:10441000C4006D00C8006D006D006D00CB00CE00C3
:10442000D100D4006D006D006D006D006D00DA00EC
:10443000DD00E000E3006D006D006D00E600E900C6
:10444000EC00EF00F200F500F800FB00FE006D004C
:104450006D0001016D006D006D006D006D000401C7
:1044600007010A01A22080E7042020817D4869E03D
:10447000000A822800D99BE0002078E7784800886D
:1044800075E700F039FA72E7FFF77CFE70E7FFF797
:104490006BFE6DE7FFF786FE6AE7CF20400064E71A
:1044A0006E48008863E7B6205FE7042020816A48F1
:1044B00048E0BC2059E76748008858E7644800880E
:1044C00055E7DE2051E76148008850E7FFF704FE1A
:1044D0004EE75D4800884AE7C02046E75948008813
:1044E00045E7DC2041E75648008840E7534800880C
:1044F0003DE7514800883AE74E48008837E74C4886
:10450000008834E74948008831E7474800882EE7AB
:1045100004202081434815E04148008827E7042013
:1045200020813E480EE03C48008820E7394800885A
:104530001DE7374800881AE73448008817E7042049
:10454000208131480068306012E72E4800880EE76D
:104550002B4800880BE72948008808E72648008890
:1045600005E76B48008802E722480088FFE62048FC
:104570000088FCE61D480088F9E61B480088F6E63E
:1045800018480088F3E616480088F0E613480088CB
:10459000EDE611480088EAE60E480088E7E60C4898
:1045A0000088E4E609480088E1E606480088DEE67F
:1045B00070BD30200621FFF70BFE70BDA401002066
:1045C000007EFFFFF20C002068110020F40C002098
:1045D000F00C0020180D00200C0D00200C11002004
:1045E000FC0C0020DA0C0020D80C0020FA1000206F
:1045F000F8100020FC100020DE0C0020DC0C002055
:10460000D60C0020D40C00200811002050110020EE
:10461000521100205E160020E00C002090010020C6
:104620008C01002088010020CE030020D003002050
:10463000CC030020F80C0020FA0C0020F60C00201F
:1046400010110020C8100020AC0D0020B00D00207B
:1046500088100020F6100020E8100020C60300207B
:10466000AE0D002048110020F0B581B0ED4EB088AD
:10467000022843D3234F8F4C234D05E02080FCF7C5
:104680003FFEB088012839D9022030813088C11915
:104690001E2919D87944097949008F441215151A31
:1046A0001D20151515151523151515151515281586
:1046B00015151515152B151515150F002868C009AA
:1046C000DCE718480088D9E7000A842816D80020BB
:1046D000D4E713480088D1E710480088CEE70C21C2
:1046E0000D4801E00A210B48FFF786FDC9E708489D
:1046F0000088C3E7A420FA49085ABFE701B0F0BD1B
:10470000A4010020007CFFFFB80F0020C0010020A2
:104710006C110020EE7E0008C27E000858110020B7
:1047200054110020BC0F002068110020F0B581B0AA
:104730001E4614460D46074600F002FDA0203043F9
:1047400000F046FD380A00F043FDF8B200F040FDED
:1047500000F0F6FCA120304300F03AFD00F0C4FC6C
:104760002870022C0AD36D1C012600F06DFC00F0AD
:10477000BBFC28706D1C761CA642F6D300F008FD29
:1047800001B0F0BD70470000B0B5541801252D03ED
:10479000AC4209D8112B03D0102B05D1044B00E0FB
:1047A000024B5918FBF7ECFCB0BDC04600100108E5
:1047B00000000108F0B581B000920E4601460E4C93
:1047C00000272760F2B210232046FFF7DDFF701E9E
:1047D00086B2A55DC1B22046FCF7CAFA854203D174
:1047E0000020A055012701E00098206003480760E1
:1047F000206801B0F0BDC04660110020C01000204C
:10480000F0B581B00446032216022A4D0423304637
:104810002946FFF78BFFAF7802212846FCF7A8FA5C
:10482000014600208F4216D129883246E732914254
:1048300011D80C2251437018C01C288080B2042368
:104840002146FFF773FFE57A0B212046FCF790FA2B
:10485000291A4842484101B0F0BDC046F0B581B0C8
:10486000044671200602134D0322042330462946D4
:10487000FFF75CFFAF7802212846FCF779FA874200
:1048800014D12888122250433018C01C288080B2CE
:1048900004232146FFF74AFF657C11212046FCF7DF
:1048A00067FA291A4842484101B0F0BD002001B022
:1048B000F0BDC04668110020B0B503F06AF8594C4D
:1048C000A28820882169C91C0423FFF72FFFA08834
:1048D000411EA18020698AB21218D578C01CC9B2C5
:1048E000FCF746FA854204D12069A1880818AA215C
:1048F000C17003F052F8B0BD0120704710B54948AF
:10490000C288511CC180036912490C789C54C2882A
:10491000531CC38003694C789C54C288531CC380C9
:1049200003698C789C54C288531CC3800369CC787B
:104930009C54C288531CC38003690C799C54C28860
:10494000531CC38003694979995406210181FEF7FC
:10495000F1FD10BD7811002010B5044600F0F0FB09
:104960003E2000F035FC204600F032FC00F0E8FB71
:104970003F2000F02DFC00F0B7FB044600F064FB84
:10498000240200F0B1FB241800F096FB00F000FCBC
:10499000204610BDF0B581B0214C2078FE21009159
:1049A00008402070812040002518FDF705FA1D4FB2
:1049B000A61C3E617D611C48205CB881FEF77EFD2F
:1049C000002814D0FEF7A4FC1848FEF72DF8B87A9A
:1049D000174960542078022101432170FCF7C0FD83
:1049E0000020144A0146FCF7EDFD01B0F0BD20782F
:1049F00000990840207000201521FCF72FFD0B4C7A
:104A00002661207840010C49421821460C3120468D
:104A1000FDF796FE2046FDF7FDFF01B0F0BDC04654
:104A2000B20D0020A401002002020000BC00002002
:104A3000030200001514000800900240F0B581B098
:104A40000A4D00242C606C60F14E2746204621461A
:104A50000A222346FBF77CFBF25D801861417F1C34
:104A60000E2FF5D103C501B0F0BDC046A81000203F
:104A7000F0B581B01A48002282831A490A601A4BA5
:104A80001C88022C04D31346022C04D20B2503E00D
:104A90000323022CFAD30825DD4EF75C0A24624377
:104AA000D2195B1C9FB2BD42F7D10A607219858B87
:104AB0000023D65C6543AD195B1C032BF9D18583BC
:104AC00008687D21CA00002421462346FBF740FBED
:104AD000AAB2064B801818606141596001B0F0BD60
:104AE000C001002098100020B0000020901000208D
:104AF00010B5C6490B780F201C090340C44A5370F7
:104B000014704B781C090340D37094708B781C0987
:104B1000034053711471CB781C090340D371947115
:104B20000B791C090340537214724B791C09034022
:104B3000D3729472C979084050730809107310BD7C
:104B400080B5054B586305481861022101221846BB
:104B5000FEF7A8FA80BDC046002C0140FDFF000012
:104B6000F0B581B000905F20C7430F4300F010FB09
:104B70000724012002F0FBFE00F0E2FAFDB2284615
:104B800000F026FB064600F003FB002E03D0601E5B
:104B9000002C0446EDD100F0D3FA284600F018FBB3
:104BA000009C200A00F014FBE0B200F011FB01B001
:104BB000F0BD0000B0B586B000F08AF8002801D042
:104BC00006B0B0BD9448002505609248058001A854
:104BD000FFF744FE00280ED08C480399C17001A94C
:104BE0004A7902708A794270CA7982704A7A02716F
:104BF000897A41713FE001A8FFF702FE002837D013
:104C0000824C0398E07001A841792170817961702C
:104C1000C179A170417A2171807A607106212046A4
:104C2000FCF7A6F8A07122780F20130902407849FA
:104C30004A700B70627813090240CA708B70A278B8
:104C4000130902404A710B71E27813090240CA71DC
:104C50008B712279130902404A720B72627913092F
:104C60000240CA728B72E2791040487310090873CF
:104C7000664885800560654C06212046FCF778F87B
:104C8000A07122780F201309024061494A700B700D
:104C9000627813090240CA708B70A278130902402F
:104CA0004A710B71E27813090240CA718B71227943
:104CB000130902404A720B72627913090240CA72E8
:104CC0008B72E279104048731009087306B0B0BDCA
:104CD000F0B587B0FFF78EFA002802D0002007B0A9
:104CE000F0BD00252E4602E0761C042C0AD2F4B258
:104CF0002046FCF7DDFD0028F6D0E8B205A90E54E9
:104D00006D1CF1E72806E9D03F4800210170EEB2A2
:104D1000012000900002039005AF019104913B4DEA
:104D200007E0394A147004900191761E7F1C002E12
:104D300020D03C780E20029060430399401807224F
:104D40002946FFF71FFD2878AA4AD070687890702E
:104D5000A8785070E87810701068297951706979D6
:104D6000117004998142E0D81188DAD1019A8A42FF
:104D7000DBD8D6E7244C207802994143039E88195A
:104D80000722224D2946FFF7FDFC2A780F20130940
:104D900002401F494A700B706A7813090240CA70BA
:104DA0008B70AA78130902404A710B71EA781309D3
:104DB0000240CA718B712A79130902404A720B7240
:104DC0006A7913090240CA728B72EA7910404873FB
:104DD000100908732078052250433018D030874ED0
:104DE0003146FFF7CFFC347904213046FBF7C0FF92
:104DF000084A00211180E971844200D131680648D7
:104E00000160009807B0F0BDC4030020E40C00204E
:104E1000740100208A100020CC100020F0B583B06F
:104E2000812080000290001F724D02222946134605
:104E3000FFF77CFC6C78012728463946FBF798FF82
:104E4000844271D17C026B480078394908531121A2
:104E5000C9431538884267D3684E07220223029857
:104E600031460192FFF762FCB57906213046FBF727
:104E70007FFF85420FD171885E4B1980B1885980C0
:104E80000021B17131882B4A118019682A4A1160BA
:104E9000854207D048E0274900220A8026490A6057
:104EA000854241D1F148005B02283FD33D463C4654
:104EB000019A57430298381880B202233146FFF70F
:104EC00035FCB77906213046FBF752FF6900194AD5
:104ED000511887420ED17288464B1A80B2885A8088
:104EE000AA001B68144EB350444E0022B27132889F
:104EF0000A8005E0AA0000230F4EB3503F4E0B80FE
:104F0000874211D1A8000C4A11581018001F0068E0
:104F1000814209D901204002D449085A641CE7B2F1
:104F2000B8423D46C4D801E0FCF768FB03B0F0BDD1
:104F3000C001002018100020C80F0020F0B581B07B
:104F40000126B0022B4D0222009029461346FFF79E
:104F5000EDFB6F7828463146FBF70AFF874207D101
:104F60002878254C20802121C9432538884213D236
:104F70002448254901812549C18025498180254949
:104F80004180002101801C48052202801C480160EC
:104F90004160018101B0F0BD20880028FAD00020D6
:104FA000164D07460BE04A000020154B9852490069
:104FB000144A50527F1CF8B221888142EAD9052256
:104FC000504300990818801C80B202232946FFF73D
:104FD000ADFB2E7904212846FBF7CAFEF9B28642C2
:104FE000E1D148002A88064B1A52002028716888AF
:104FF000DDE7C04668110020C40F002060110020CA
:10500000640D00201A0D0020204E0000983A000088
:10501000102700008813000009490988022908D0D8
:1050200001290BD107490988002907D1C01C80B28A
:10503000704704490988012900D1C01C80B270471B
:10504000B2000020B0000020F0B581B07F4C1025E8
:105050000026204629463246FDF72BFE00BF40348D
:105060000127204639463A46FDF723FE00BF204679
:1050700039463246FDF71DFE00BF744829463A46C0
:10508000FDF717FE01B0F0BD70B5704C25464035F8
:1050900000212846FCF78FFB04212046FCF78BFB00
:1050A0000126284631463246FDF703FE10212046F0
:1050B0003246FDF7FEFD70BDB0B50A4C20464038C3
:1050C000102101252A46FDF7F4FD00BF20462946A0
:1050D0002A46FDF7EEFD00BF002220462946FDF7D7
:1050E000E8FDB0BD80080140F0B581B0574804210B
:1050F000FCF758FB002508240095544F3D464035E9
:105100000126284631463246FDF7D3FD00BF102167
:105110003846FDF7C7FD0746002228463146FDF711
:10512000C8FD781E874100984000C51900BF641E65
:10513000E2D104214548FCF73EFBE8B201B0F0BDE6
:10514000F0B581B0414E3446403400252046294612
:10515000FCF731FB04213046FCF72DFB102601271C
:105160003A4831463A46FDF7A4FD204639463A46CC
:10517000FDF79FFD354831462A46FDF79AFD00BFF1
:10518000204639462A46FDF794FD01B0F0BDC046E1
:10519000F0B581B02D4E4036012500273046294616
:1051A0003A46FDF786FD00BF1024284821463A46BE
:1051B000FDF77FFD00BF304629462A46FDF779FD01
:1051C000224821462A46FDF774FD01B0F0BDC046D5
:1051D000F0B581B006460824F0B2C20910211B4D7B
:1051E0002846FDF766FD40350127284639463A46F0
:1051F000FDF75FFD00BF002228463946FDF759FD47
:1052000000BF641E7600002CE6D104210F4E30460C
:105210000C46FCF7C7FA0127284639463A46FDF7FF
:1052200048FD00BF10213046FDF73CFD0646002238
:1052300028463946FDF73DFD04482146FCF7BBFAF8
:10524000701E8641304601B0F0BDC04640080140A6
:1052500080B5FCF7D9FB80BD80B5602003213C22DE
:10526000FFF7A8FADE21E44A505280BDC0010020B9
:10527000F0B581B0494F3878002800D18CE0032880
:105280001FD1474F552038700126B2024548464984
:10529000FAF776FF454D464C284629462246FDF74B
:1052A000D5FB002800D0FEE732023E4928462346BF
:1052B000FDF722FC002800D0FEE700203870374FB1
:1052C00038700125AA02374C38492046FAF758FFB2
:1052D000384801782322A1542146233182788A70EC
:1052E00040784870BC21E148415A21842146203150
:1052F0000246BC3292788A70018821874188618792
:105300008188A187C188E18701894022A152408913
:1053100042216052387801280BD0022838D1234E20
:10532000234C304631462246FDF790FB00280AD038
:10533000FEE71E4E1E4C304631462246FDF786FBE8
:1053400000280AD0FEE72D02164930462A46234699
:10535000FDF7D2FB002809D0FEE72A0211493046AA
:105360002346FDF7C9FB002812D0FEE70E4E30465B
:1053700031462246FDF76AFB002800D0FEE70949C6
:1053800030462A462346FDF7B7FB002800D0FEE74B
:10539000034800210170397001B0F0BDF510002004
:1053A000F4100020981100200000010800100108EE
:1053B000FFFFFF00F6100020B0B58C4DA87A000169
:1053C0008B4C607169782A78120189182170E9780C
:1053D000AA7812018918617069792A7912018918ED
:1053E000A170E979AA7912018918E170697A2A7A9B
:1053F000120189182171E97A081860710621204686
:10540000FBF7B6FCA071687B297B09014018E071AD
:10541000B0BDC04670B5A34903220A767E4A002378
:10542000138004240C818C88032C01D88B8070BDE0
:1054300005240C76304C2468304DAC4205D0304DFC
:10544000AC4202D02F4DAC421CD12F4C23800B76A6
:1054500001231380CA88551CCD800B699E5CEE4CDD
:10546000E670961CCE80ADB25D5DA570D51CCD807A
:10547000B6B29E5D6670121DCA80A9B2595C2170D9
:105480002168016070BDC046014802490180704733
:10549000BC100020FFFF000070B5824903220A768D
:1054A0005D4A0023138002240C818C88012C01D8D2
:1054B0008B8070BD05240C760F4C24680F4DAC42D8
:1054C00005D00F4DAC4202D00E4DAC4212D10E4C65
:1054D00023800B7601231380CA88531CCB800C6970
:1054E000A55CCD4E7570921CCA8099B2615C31701A
:1054F0003188018070BDC0464811002055AA0000C7
:105500004452495333313032A2010020F0B581B00A
:1055100034480024048034480460344E7078317874
:1055200009014018324D2870F078B178090140180F
:1055300068707079317909014018A870F079B179F3
:1055400009014018E870707A317A09014018287111
:10555000B07A0001F17A0818687106212846FBF735
:1055600007FCA87123490C6040488483727B337B1D
:105570001B01D218EA71214A1388022B04D3224658
:10558000022B04D20B2503E00322022BFAD30825B9
:10559000B75C0A235C43E419521C97B2BD42F7D1B1
:1055A0000C607119002216468D5C5E437619521C00
:1055B000032AF9D186837D20C20000252046294692
:1055C0002B46FAF7C5FDB2B20D4B80181860694141
:1055D0005960FCF7A9F9681C042D0546F9D301B000
:1055E000F0BDC0468A100020CC10002074010020BD
:1055F000E40C002098100020C0010020B000002022
:1056000090100020062803D3034800220280084699
:1056100040000249085A7047FE100020F87E00083A
:1056200080B507480021C160016141720321C17149
:1056300081888279120489180068FBF73DF980BDE2
:105640001411002010B5194C2078FC210140217064
:10565000A4200649085A800005490858FBF70CFFAA
:105660002078FE210140217010BDC046C0010020FD
:10567000EC98000880B50A48FDF7D6F90948807A09
:1056800009490A4A50541078022101431170FBF76E
:1056900067FF0020064A0146FBF794FF80BDC04625
:1056A000BC000020A401002003020000B20D002075
:1056B0001514000870B582B004460F4D2846FDF75A
:1056C00057FB01AE00203070FDF71EFC10207080EB
:1056D0000220707028463146FDF76CFB01262846F3
:1056E0003146FDF759FB70073749086028462146C7
:1056F000FDF794FB02B070BD000C0040F0B581B026
:1057000004466E460020307001252846FDF7FCFB5C
:105710001020708002207070084F38463146FDF727
:1057200049FB38462946FDF737FBA806264908609D
:1057300038462146FDF772FB01B0F0BD200C004059
:1057400080B50A480178FE220A4002700120C00399
:1057500000F014F86248064900F0CCFE054800212C
:10576000018005480180FCF74FF980BDA0010020B1
:1057700051520008061100200411002070B582B0BB
:105780000546002601960F480090554C6946204674
:10579000FDF794FC656366620221012520462A46D6
:1057A000FDF780FCE80608490860FF20000607496D
:1057B0000A688243A807101808602046FDF7AAFC73
:1057C00002B070BDF400FFFF00E100E018E400E06B
:1057D00010B51048C089504C20807120032102F080
:1057E0001BF8294908800D48417802220A4342707B
:1057F0002348417809024C3101800948814208D18F
:10580000002020800A20022102F006F82080FBF709
:10581000FBFF10BD1C16002068110020BC0F0020EB
:105820004C48000070B5164D0020288071200321DF
:10583000144C2246FEF7BEFF13490880144E31680F
:10584000002908D0114908409634A04203D2288884
:105850004C2101432980742003210E4AFEF7AAFF40
:105860000D4908803168002908D080B20B49884270
:1058700004D30920C00229880143298070BDC04695
:105880005C1600201027000052110020FEFF0000CF
:10589000C010002004290000501100209F39000092
:1058A00080B5012800D00220FCF76EFE80BD00000C
:1058B000B0B50B4C2046FDF733FC0120C00609496A
:1058C0000860BFF34F8FBFF36F8F472520462946EF
:1058D000FDF7E4FB002220462946FDF7E3FBB0BDBF
:1058E000002C014080E100E010B58100094A5158C8
:1058F000094A1160094B59804100094C615A1980CD
:10590000518899800721484381229200801801F034
:105910005FFF10BDC80F002068110020601100203B
:10592000181000200348007803490A68101808601E
:105930007047C046140000209411002080B584B048
:1059400000200390029008200190042000906846F7
:105950000349FDF769FA002800D0FEE704B080BDD6
:10596000FFFF000080B582B01C4908680007800F67
:1059700000905A48009A032A0BD8C0467A441279FC
:10598000520097440104080B0A68520401D4144AD7
:1059900006E0019005E07D22120201E00122D2031F
:1059A000019209680906090F00910099082901D29E
:1059B000002106E0009A00990B2A01D8C91F00E0D7
:1059C000891F00910199009AD140434A11601168E2
:1059D000FDF778F94249087002B080BD041002401A
:1059E0000048E801B0B582B06C460020A071FF20ED
:1059F0000230A0800B4800900B4D28462146FDF751
:105A0000CDF8284640302146FDF7C8F820881E21F1
:105A100088432080803528462146FDF7BFF802B034
:105A2000B0BDC046FFFF010000080140F0B581B0E5
:105A30007F4800240460214F3C808480022520465A
:105A40002946FEF75FFB401CC6B2204631462A4677
:105A500001F0B6FD20462946FEF754FB864205D0EC
:105A60000120734948707978014379700024042536
:105A700020462946FEF746FB401CC6B2204631466A
:105A80002A4601F09DFD20462946FEF73BFB864253
:105A900005D0012066498870797801437970062025
:105AA000FEF75AFF542806D00120614948717878E2
:105AB00040210143797001B0F0BDC046561100206D
:105AC0000548064901600648022101700548016841
:105AD00001220A4302607047100000200024F400F5
:105AE0000000002014100240F0B581B0494C20881D
:105AF000494DA8426FD04948002606804848008892
:105B0000411E88414001474FB9892022914308181E
:105B1000B88101F02BFF44480660444806804448A1
:105B200006604660866043484021FAF750FBA42097
:105B300005213952A22001213952A0203E529E2037
:105B40003D493952572080003E52B6203E52B8207F
:105B50003E52BC203E5239480660394806603948FA
:105B6000066039480660394806803846BC304680B1
:105B70008680C680068136480178DF220A4002709E
:105B800034480178FA220A40111D0170DA203E5291
:105B9000D8203E52C8203E52CF2040003E52C12065
:105BA00040003E520320C0013E522B4806602B4865
:105BB00006602B4806602B4806602B4806802B4861
:105BC000066046602A4806802A4806702A480178FE
:105BD00010220A430270FFF757FAFBF781FD1D48B8
:105BE000417806220A4342700120010201F0AAFE18
:105BF000FFF71CFF00F044F8A4200A49085A80006F
:105C00001E49085800F09AFCFFF71CFD258001B0E2
:105C1000F0BDC0465A11002055AA0000C410002053
:105C2000B6000020C0010020A0100020421000207B
:105C3000640100201C16002025200000F010002028
:105C4000E8100020EC100020E41000208810002054
:105C5000BC0F0020A001002098150020000D00209E
:105C6000080D0020040D00208A1000209010002054
:105C700090110020F510002040100020EC98000842
:105C8000F0B583B0FD4C2078BF2101402170FFF7B3
:105C9000C9FDFB480188FB48018021780A07FA4EBC
:105CA00010D4CA0719D000220280DF2001402170E1
:105CB000F648017804220A430270F5480188314011
:105CC00001800AE000210180F14801883140018013
:105CD000EE48017804220A43027000252846FCF7AA
:105CE000DFF8EC490A68904201D0EB4A1560086081
:105CF00020781421084205D0E54801883140018010
:105D0000052006E0E5480088002801D0022000E0D8
:105D10003C20E34C2560E349088036210222102311
:105D20002046FEF731FD6778012620463146FBF715
:105D30001FF8874202D10020607001E025602E46E6
:105D4000D948066020682560D84908803821022299
:105D500010232046FEF718FD6678012520462946C7
:105D6000FBF706F8864202D10020607001E00025B2
:105D70002560CD480560206800262660CB49488014
:105D80003A21022210232046FEF7FEFC6778012507
:105D900020462946FAF7ECFF874202D100206070C6
:105DA00001E026603546C048056020682660BF498E
:105DB00088803C21022210232046FEF7E5FC66780D
:105DC000012520462946FAF7D3FF864202D100205A
:105DD000607001E000252560B3480560206800265A
:105DE0002660B249C8803E21022210232046FEF7D9
:105DF000CBFC6778012520462946FAF7B9FF874290
:105E000002D10020607001E026603546A64805609A
:105E100020682660A54908814021022210232046DF
:105E2000FEF7B2FC6678012120460291FAF7A0FF46
:105E3000864203D100206070012001E00020206034
:105E400099490860206800262660984948811421F5
:105E5000032210232046FEF797FCA7780221204654
:105E6000FAF786FF874203D10020A070012003E0EB
:105E70007D20C000206030468B4908602068266085
:105E80008B4908804821052210232046FEF77CFC20
:105E9000267904212046FAF76BFF864203D10020C1
:105EA0002071012001E0002020607F490860206807
:105EB000002626607F4908604D21032210232046DA
:105EC000FEF762FCA77802212046FAF751FF8742CD
:105ED00003D10020A070012004E07D20C0001E300E
:105EE000206030462168B622704B99526E49086096
:105EF00026605021052210232046FEF745FC267916
:105F0000042120460191FAF733FF864203D1002095
:105F10002071012001E000202060634908602068B2
:105F200065490860FAF748FF01F020FD0026266069
:105F30002321032210232046FEF726FCA578022108
:105F40002046FAF715FF0299CF03854203D10020BE
:105F5000A070012001E027603046F2490860206807
:105F60002660F24908802021032210232046FEF7F4
:105F70000BFCA57802212046FAF7FAFE854203D1F0
:105F80000020A070012001E0276000202168BC22D1
:105F9000E54B9952E349086000262660B6210322AA
:105FA00010232046FEF7F0FBA57802212046FAF7E1
:105FB000DFFE854204D10020A070D94F029902E093
:105FC00027603146D64FD748016020682660D849FF
:105FD00008802621022210232046FEF7D5FB667892
:105FE000012520462946FAF7C3FE864202D1002049
:105FF000607001E000252560CA480560208838806F
:10600000CC49088000273946FFF7FCFACA21C64A66
:1060100050522760F621022210232046FEF7B4FBDF
:106020006678012520462946FAF7A2FE864203D16A
:1060300000206070012002E0019820603846B949D4
:1060400008602088BC49088004263146FFF7DAFA48
:10605000BA21B54A50522760282105221023204634
:10606000FEF792FB277920463146FAF781FE8742F8
:1060700024D100202071012023E0C046BC0F002065
:106080008810002044110020FFBF0000A001002064
:106090004011002098150020CC100020C2030020E1
:1060A000601100206E110020C0100020C0010020EF
:1060B000C603002088010020900100209F48206036
:1060C0000020984908602068002626609C490860E6
:1060D000F821052210232046FEF756FB27790421DC
:1060E0002046FAF745FE874203D1002020710120A7
:1060F00001E0266030468B4908602068266091499F
:1061000008602D21032210232046FEF73DFBA678D0
:1061100002212046FAF72CFE864203D10020A0700F
:10612000012002E08848206000207E490860206845
:10613000002626608549088042210322102320463C
:10614000FEF722FBA77802212046FAF711FE8742CC
:1061500002D10020A07002E07D48206035467148E1
:106160000560206826607B4908801C2102221023DC
:106170002046FEF709FB6578012620463146FAF7EE
:10618000F7FD854203D100206070012001E000206E
:106190002060644908602078002727606E490880E5
:1061A00045210322102320460292FEF7EDFAA5783E
:1061B00002212046FAF7DCFD854202D10020A070C2
:1061C00002E0962020603E465648066020686349FB
:1061D000088001F0CBFB27601E21022210232046FD
:1061E000FEF7D2FA6578012620463146FAF7C0FD5F
:1061F000854203D100206070012002E002982060F7
:1062000000202168DC22484B99524649086000254D
:106210002560E921032210232046FEF7B5FAA7786E
:1062200002212046FAF7A4FD874202D10020A07087
:1062300002E0302020602E462068EC21EC4A5052CB
:10624000384806602560022210232046FEF79CFA9B
:106250006678012520462946FAF78AFD864203D151
:1062600000206070012002E01A20206000202268D7
:10627000EE21DF4B5A522B4A106000262660032283
:1062800010232046FEF780FAA77802212046FAF76D
:106290006FFD874203D10020A070012001E026603D
:1062A00030462168F022D24B99521E49086001F015
:1062B0005DFB00F07BF9FDF77BFEFBF785FCFEF74D
:1062C000CBFFFAF775FBFEF7A9FDFEF737FEFEF7E9
:1062D00071FCFFF7D9F8FBF7FDFDFAF7A3FD266087
:1062E0001F49032210232046FEF74EFAA67802210A
:1062F0002046FAF73DFD864202D10020A07002E060
:10630000642020600025074805602088154C208007
:10631000FBF7ACFF002801D06420208003B0F0BD63
:1063200088100020C0100020C0010020F6100020BE
:10633000FA100020421100200E110020C027090091
:10634000E8100020F010002010270000AC0D002005
:10635000B80B000010110020C81000205E160020AD
:10636000AE030000180D0020B0B534480078AA280C
:1063700001D1FEF77DFF32480078C00720D03148B8
:10638000034614330ECB304CA1812283E382416A51
:10639000826A2181E281008C2C494140E18388B2EC
:1063A0000021FBF763FC2A4901250D70FAF709F972
:1063B00028490860E0892849884201D327480570A8
:1063C00027480078C00701D0FEF7E4FA2348007898
:1063D000401E4142414123480078401E4242424112
:1063E0000A43012A1ED19D49087800280BD00020BD
:1063F00008701E490A78521CD3B2032B00D81046ED
:10640000087000F02DF912480178002914D00021FD
:10641000017000F025F9164C207800280CD1FAF70D
:10642000CFFB07E0104C2078002805D1FDF7D0F80D
:10643000FDF714FA01202070B0BDC046F410002012
:10644000A0010020141100201C1600200080FFFF76
:10645000441000200011002051C3000092110020C0
:10646000B20D0020B2100020E20C0020BE0F002070
:10647000B1100020B0B5064C2568A80704D5254802
:106480000068002800D080470948A8432060B0BDBC
:10649000102C0140B0B521480068044C2568002844
:1064A00000D080470248A8432060B0BD10000040E3
:1064B000FFFF000010B506480068002800D08047A4
:1064C00001242046FCF702F92046FCF795F810BDA0
:1064D000100D002010B506480068002800D0804745
:1064E00002242046FCF7F2F82046FCF785F810BDA0
:1064F000140D00200122084B984205D093079842C2
:1065000007D11007054A01E0D006024A044B186083
:106510001160704770110020002C014074110020A0
:1065200000E100E010B5194C04212046FCF700FE04
:1065300002212046FCF7FCFD10BDC046F0B587B037
:10654000019005AD0327AF7101200002A8800D481E
:1065500005903F4E30462946FCF720FBAF710024E2
:10656000AC800948059030462946FCF717FB02A984
:106570000C810397019802900448FCF7EFFD07B0E7
:10658000F0BDC046020000010400010100380140D6
:1065900010B5054C04212046FCF7CAFD0221204617
:1065A000FCF7C6FD10BDC0460048004010B51A20DB
:1065B000022421462246FEF7FDF8C0210C4A505223
:1065C000401E83B2032B06D200B241000948405A54
:1065D000094A545A01E05452204608490C8008499F
:1065E0000C8008490880084908800849088010BDC7
:1065F000C00100208C7D0008867D00089C100020D2
:106600009E100020B4000020B2000020B000002046
:1066100010B50F4801242146FCF744FB0D490A78C8
:10662000002A04D0012811D1002008700BE00028B6
:1066300009D109480288521C028090B2032805D370
:10664000064804700C7004480021018010BDC0464B
:1066500000080140EE0C0020EC0C0020C6100020C9
:10666000F0B58BB0AD480068FAF70CF80025AC4BDC
:106670002A46F9F723FF07460E46AA480478012C5C
:1066800007D0022C08D0032C0ED101208207A74B83
:1066900004E00022A64B01E00022A34B384631461D
:1066A000F9F7A4FE07460E46032C24D87C4424792F
:1066B0006400A7440128496B05204207A54B3846D2
:1066C0003146F9F7E1FDF9F79FFF0A900024A24B4C
:1066D000384631462246F9F789FE994B2246F9F7AA
:1066E000D3FDF9F791FF0A21F9F7E0FF0591662044
:1066F00008909BA025E07E2008908E480490059588
:1067000009950A9563E005204207924B38463146C9
:10671000F9F7BAFDF9F778FF0A9000248E4B384656
:1067200031462246F9F762FE854B2246F9F7ACFD69
:10673000F9F76AFF0A21F9F7B9FF05915A20089085
:1067400086A00490012041E0072042077A4B38469A
:106750003146F9F799FDF9F757FF0A900024704B7D
:10676000384631462246F9F741FE754B2246F9F785
:106770008BFDF9F749FF7D21C900F9F797FF0591D6
:106780004E20089071A0049003201FE007204207CC
:10679000694B38463146F9F777FDF9F735FF0A902E
:1067A0000024664B384631462246F9F71FFE644BFB
:1067B0002246F9F769FDF9F727FF6421F9F776FF1B
:1067C00005914E2008905FA00490022009900126B8
:1067D0000A980028354609D000260A9C0A2120463E
:1067E000F9F764FF761C092C0446F7D8002014271B
:1067F0007E222C23039039460797FCF7F9FE00957B
:106800000695182408983946049A2346FDF7CBFAD2
:10681000009401950B20C04301467143099A5043EF
:10682000089A871808970C3FC819C0B2F3B2079DA1
:1068300029460A9AFDF778FA069E0096F8B22E22AB
:1068400029462346FDF7E4F9009401960898C0B262
:106850002946059A099BFDF767FA4248C0894249D3
:10686000884201D904240FE04049884201D9032419
:106870000AE03F49884201D9022405E03D498842A7
:1068800001D8039C00E00124682000217E220C2313
:10689000FCF702FF692001217D220B23FCF7D2FEC9
:1068A000601E03281ED8C046784400794000874403
:1068B000130D0701792002217C220A23FCF7ECFE4C
:1068C0007420022177220A23FCF7E6FE6F200221C2
:1068D00072220A23FCF7E0FE6A2002216D220A23BD
:1068E000FCF7DAFE7E200324802209232146FCF7F0
:1068F000D3FE0020FDF788F80120FDF785F802207F
:10690000FDF782F82046FDF77FF80420FDF77CF8BC
:106910000520FDF779F80BB0F0BDC046001100204E
:1069200000408F40BE0F0020FDB87E3FE17A843FDB
:10693000A7001E40049900084D62403F00005940E6
:106940000000E03F6D62617200000000746F7272BF
:10695000000000009999A93F000024406D636D007C
:10696000706100001C160020D8AE00007DAA000057
:1069700023A60000C9A10000F0B581B07A487B4D84
:106980000560AD4C2288FF203230824235D27849F2
:106990001BE05A005219603A12880A80E288531CA0
:1069A000E38023694E789E54E288531CE380236978
:1069B0000E789E54022222812288521C2280A388B3
:1069C0009B1EA38093B2834217D2A388022B00D2CE
:1069D000C7E093B292B22F2ADBD85A005219012392
:1069E0005B02D35A23811A46303A92B20646303EB1
:1069F000B6B2B242CDD30022CFE7A088022800D29F
:106A0000AFE05D4F5A4E05E0FCF794FDA0880128E9
:106A100000D8A6E0022020812188C8193C2800D98E
:106A20005DE0C0467844007940008744671E7733B4
:106A30001E77331E77331E77331E77331E77331E50
:106A400077331E77331E77331E77331E77331E77E7
:106A5000331E77331E77331E77331E77331E77331B
:106A60001E77331E77331E773300042020810120E8
:106A700040022A5A3F484018801C80B2404948438F
:106A8000400C824201D80021316080003E49085804
:106A9000306010E0012040022A5A3648081880B2BF
:106AA00037494843400C824201D8002131804000E0
:106AB0003449085A30802089002800D1A4E70121F8
:106AC000E288531CE3808BB280B2C01A305C236929
:106AD00098542089491C8AB29042F1D294E7274801
:106AE000081805281AD8C046784400794000874421
:106AF00002090B0E10134B20C000DBE701204002FF
:106B0000285AD7E71A20D5E77D200001D2E71220C6
:106B1000D0E77D20C000CDE70C20CBE71B48084024
:106B200020800F2212030A40228101210B039A4286
:106B300009D003231B039A4208D049038A4210D18B
:106B40001449122206E012491A2203E04B21C9001F
:106B5000AB310C22424350182080FDF7ADFE0020DF
:106B6000A08001B0F0BDC04660010020C00100203F
:106B700068110020CDFE0000D0FEFFFF00F1FFFFF6
:106B8000ABAA000018100020C80F0020FF0F000063
:106B90000331000003710000F0B59FB0264F7888E4
:106BA000012105910C0221466D31884202D9022053
:106BB000387623E021490968002206E006AEB55286
:106BC0005B1C3B80921C662A0ED03B8883420BD212
:106BD0002F2B1D46F2D85D006D1801267602AD5BA5
:106BE0003D81302DEAD0E2E715480078002802D038
:106BF000144815490160387E002801D01FB0F0BD4F
:106C0000032004900002039002E0387E0028F5D1B2
:106C1000FCF7A4FC0028F1D13888400006A9095AE5
:106C20000A46373A53089A2B00D9BEE107A352000F
:106C30009A5A52009744C046A401002060010020E7
:106C4000BE1000204811002055AA0000B401B9016F
:106C5000B901B901B901BF01B901D401B901B90143
:106C6000B901B901B901B901B901B901B901B90154
:106C7000B901B901B901B901B901B901B901B90144
:106C8000B901B901B901B901B901E601B901B90107
:106C9000B901B901B901B901B901B901B901B90124
:106CA000B901B901B901B901B901B901B901B90114
:106CB000B901B901B901B901B901B901B901B90104
:106CC000B901B901B901B901B901B901B901B901F4
:106CD000B901B901B901B901B901B901B901B901E4
:106CE0004402B9015502B9016602B901B901B901FD
:106CF000B901B9017502B90186029A02B901A4026B
:106D0000BA02C502D002E002EB02B901B901B90131
:106D1000B901B901B901B901B90100030B03B90106
:106D2000B901B901B901B901B901180323032E034F
:106D3000B901B901B901B901B901B901B901B90183
:106D4000B901B901B901B901B901B901B901B90173
:106D5000B901B901B901B901B901B901B901B90163
:106D6000B901B901B901B901B901B901B901B90153
:106D7000B901B901B901B901B901B901B901B90143
:106D8000B901B901B901B901B901B901B901B90133
:106D9000B901B901B901B901B901B901B901B90123
:106DA000B901B901B901B901B901B901B901B90113
:106DB000B901B901B901B901B901B901B901390381
:106DC000B90149037403B9018C03B901B901B901CF
:106DD000B901B901B901B901B901B901940340017F
:106DE000400140014001400140014001400140019B
:106DF000400140014001400140014001400140018B
:106E0000400140014001400140014001400140017A
:106E1000400140014001400140014001400140016A
:106E2000400140014001400140014001400140015A
:106E30004001400140014001400140014001C003C8
:106E40006001B90187016001B90187016001B901E1
:106E500087016001B90187016001B9018701600103
:106E6000B90187016001B90187016001B90187019A
:106E70006001B90187016001B90187016001B901B1
:106E800087016001B90187016001B90187016001D3
:106E9000B90187016001B90187016001B90187016A
:106EA0006001B90187016001B90187016001B90181
:106EB00087016001B90187010C48411833313981DC
:106EC00088B240000A4A101A0D2252018018094A5D
:106ED000106000220092049A5143039BC91889B2A2
:106EE000234600F0B9FC022038818EE6CDFE00007A
:106EF000C00100206001002005984002FD4A105AA0
:106F0000FD4A5118891C89B2FC4A4A43550CA842D3
:106F100000D873E6FA4E3046FEF77CFAF94800884E
:106F2000002800D16AE6A8003168F74A1150F748F6
:106F300000210180F6480178F7220A400270E8B289
:106F4000FEF7D2FC61E605984002EA4A105AEA4A86
:106F5000891889B2E94A4A43550CA84200D84DE63F
:106F6000EC4E3046FEF798FAE6480088002800D13B
:106F700044E63088E84A1118703989B2914200D24B
:106F80003CE66900E54A5052E04800210180E8B241
:106F9000FEF7AAFCDE480178F7220A40027034E6C8
:106FA000F9480E30FEF778FA2FE6022038810020EB
:106FB000F849088029E6B988042900D21EE606A906
:106FC000401840883D2800D018E6F04E3046FEF7C5
:106FD00021FA3068F049884200D93AE2002039E2CB
:106FE000CF204600E84DA819FEF756FAE848018878
:106FF00048424841A95B039AE732914200D9F3E144
:107000000021F2E1B988082900D2F7E506A9411864
:107010004988572900D0F1E506A9411889885829DF
:1070200000D0EBE506A94018C088592800D0E5E556
:10703000D64E3046FEF7EEF9D84D2846FEF7EAF96F
:1070400008203881D2480088002800D1DDE5316869
:107050002E681720D24A921B884100D2D5E57D20A8
:10706000C200002302933046F9F742F8CD49086088
:10707000CD4941438919C44A9183CC4D0822012648
:1070800029463346FAF718F9BF48808B08350322A2
:1070900029463346FAF710F9029D2846FDF7BCFF52
:1070A0000646BE480660C24845730573C57280191E
:1070B0000B22BE49F9F764F80B36B8480660F5E1D3
:1070C00001200090B048A23012210222F723FAF7E3
:1070D00043FDAF480088002800D196E5F9F726FE69
:1070E00093E506A940184088842800D086E5B14879
:1070F0000068002100914308B548F821052200F0FE
:1071000097FA82E506A940184088862800D075E5E0
:1071100000200090A74828210522AE4B00F088FAF5
:1071200073E5FA2000909848B6304D210322AA4B0F
:1071300000F092FB96480088002800D165E5F9F739
:107140003BFE62E5CF2046008F4DA819FEF7A4F95B
:107150008F480088002800D157E5AA5B9F4908881E
:10716000904200D0A8E100210120B4E19C480090A9
:107170008548BC30202103229A4B00F06DFB44E58A
:10718000CF204600804DA819FEF786F98048008878
:10719000002800D139E5A85BC021695A884201D195
:1071A000FFF733FDF9F760FEFFF72FFDF54800907C
:1071B000F748C23089210322F34B00F04DFBFFF763
:1071C00024FD00200090F248C4308C210322F74BAC
:1071D00000F042FBFFF719FDCF204500EC4E70197F
:1071E000FEF75AF9EB48008841424141705B0328A1
:1071F00000D91AE1002219E100200090E448C830CB
:1072000066210222012300F027FBFFF7FEFCCF20BE
:107210004600DF4DA819FEF73FF9DE480088002838
:1072200001D1FFF7F2FCAA5BDC490888904200D04C
:1072300072E1002105987EE100200090D448DC3006
:107240001E210222042300F007FBFFF7DEFC0020D2
:107250000090CF48DE3005994B02D03360210322E5
:1072600000F0FAFAFFF7D1FC30200090C848EC306B
:10727000E9210322F02300F0EFFAFFF7C6FC05989E
:107280000090C348EE30EC210222282300F0E4FAFB
:10729000FFF7BBFC00200090BD48F030EE21032238
:1072A000BD4B00F0D9FAFFF7B0FCCF204500B84E37
:1072B0007019FEF7F1F8705BB449884201D0FFF70E
:1072C000A4FCF9F76BFDFFF7A0FCCF204500B04E02
:1072D0007019FEF7E1F8AF480088002801D1FFF7E8
:1072E00094FC705B012801D0FFF78FFCF9F758FD83
:1072F000FFF78BFCC0010020CDFE0000ABAA000010
:1073000080110020FE100020C80F0020A2010020E4
:10731000A0010020681100200BE7000018100020D9
:10732000CF2045009A4E7019FEF7B6F8E84800885D
:10733000002801D1FFF769FC705B022800D11CE135
:10734000012801D0FFF761FC00F0CCF9FFF75DFCEC
:10735000CF204000F3490818FEF79EF8FFF755FCD0
:10736000CF204500EF4E7019FAF7D4FB715BDB4874
:10737000814201D0FFF749FCD94900220A80D64951
:107380000860FFF742FCC046C001002080110020C9
:10739000FE10002068110020FFE0F5058411002098
:1073A000FFE776489810002018FC000064010020D8
:1073B00074010020E8100020049800900598410214
:1073C000D84840180222142300F046FAFFF71DFCAB
:1073D000F0100020FFFFFF7F7C150000F87E000802
:1073E00060700000A08F00000121084301D0FFF76A
:1073F0000CFCFDF77DFB2946704D00206873287357
:10740000E872885B6C4E3146083103220123F9F79C
:1074100053FF0820FDF700FE317A29542918727AAB
:107420004A70B27A8A70C01C3EE00122114301D03A
:10743000FFF7EBFBA74908806320032100F0C8F9A0
:10744000C62170525748002101605748C171FFF7AB
:10745000DCFB01209E4909884A424A41024301D08F
:10746000FFF7D3FBFDF744FB3068534E082201239E
:107470003146F9F721FF514D0020A870687028703F
:10748000FDF7CAFD317829542918F279CA71B27909
:107490008A7172794A7132790A71F278CA70B27857
:1074A0008A7072784A70083042490860FEF72EF8F8
:1074B000FDF7DEFAFFF7A9FB8B1C0020C14304296E
:1074C0000BD09D1C491C1B8893422B46F7D10529E4
:1074D00000D20120491C002803D100207C490880EB
:1074E0000421904881537A480088002801D1FFF791
:1074F0008CFBD8480180F620022100F08DF92C4940
:107500000880062803D30020714908800420400029
:107510002249085ABA212CE08B1C0020C1430429BF
:107520000BD09D1C491C1B8893422B46F7D1052983
:1075300000D20120491C002802D10021E848018026
:1075400078488153E6480088002801D1FFF75DFBA9
:10755000E44801802620022100F05EF910490880ED
:10756000062802D30020DE49088040000B49085A53
:10757000CA216C4A5052FFF748FBFAF73FF8FFF771
:1075800044FBC0466868000088B6000055AA0000A9
:10759000C0010020FE100020C8AF0000F87E0008E7
:1075A00088100020CC100020E40C0020FFFF000019
:1075B0000E110020841100206401002074010020BD
:1075C000F0B581B015460E4607467F4820210022BF
:1075D000FBF76FFB5F20C4432C43FDF7B1FDE5B221
:1075E0002846FDF7F5FD380AFDF7F2FDF8B2FDF784
:1075F000EFFD3046FDF7ECFDFDF7CAFD0727012042
:1076000000F0B5F9FDF79CFD2846FDF7E1FD0646C3
:10761000FDF7BEFD002E03D0781E002F0746EED1E9
:10762000202101226848FBF744FB01B0F0BDC046B1
:10763000F0B583B0BF4D03242C76A94C00262680DC
:1076400004242C81AC88032C02D8AE8003B0F0BD9A
:10765000009101920290E888411CE9802A69145C3B
:107660006C4FFC70841CEC8089B2515CB970C11CF9
:10767000E980A4B2145D7C70001DE88088B2105CC3
:10768000387005202876984800689849884205D0C7
:107690009749884202D09749884216D19648068079
:1076A0002E763868984210D8089988420DD30299EE
:1076B00009687960884208D00120894908800098CB
:1076C000019900F085F80299086003B0F0BDC0464A
:1076D000FE100020601100204811002055AA000073
:1076E000A2010020F0B581B00D2040010D4908181D
:1076F0000D4C206000250D4E8F4F705D2168088075
:1077000038800321084668430A02801880B200F0DE
:107710005FF82068801E20606D1C302DEDD101B017
:10772000F0BDC046C001002060010020927E00082C
:10773000F0B583B0029300920C4606462248202101
:1077400000273A46FBF7B5FA5F20C5430298054388
:10775000FDF7F6FCE8B20190FDF73AFD300AFDF7BF
:1077600037FDF0B2FDF734FD0098002810D0054633
:1077700003E0641C7F1CAF420AD22078FDF728FD8D
:10778000761CB006F5D1B0B20299FDF7E9F9F0E741
:10779000FDF7FEFC0726019D012000F0E8F8FDF74B
:1077A000CFFC2846FDF714FD0446FDF7F1FC002C44
:1077B00003D0701E002E0646EED120210122024881
:1077C000FBF777FA03B0F0BD4008014070470000B6
:1077D000F0B581B00D4604464E1EF1B20D4F38464D
:1077E000F9F7C6FAB2B200923946B85402272046D9
:1077F0002A463B46FFF79CFF002606490E602046BE
:107800000C462A463B46FCF791FF00982654206818
:1078100001B0F0BD60110020F0B581B00D46044606
:107820004E1EF1B2444F3846F9F7A2FA3946B85520
:10783000022720462A463B46FFF77AFF20463E4C69
:1078400021462A463B46FCF771FF0020A0552088C0
:1078500001B0F0BD68110020F0B583B0354D0324B0
:107860002C761F4C0026268002242C81AC88012C0B
:1078700002D8AE8003B0F0BD009101920290E8887A
:10788000421CEA8029690C5C2B4F7C70801CE880CC
:1078900090B2085C387005202876134800681349B8
:1078A000884205D01249884202D01249884215D137
:1078B000114806802E76388898420FD80899884259
:1078C0000CD302990988884208D001200449088015
:1078D00000980199FFF7A0FF0299088003B0F0BD5E
:1078E000FE100020681100204811002055AA000059
:1078F0004452495333313032A2010020F0B50D4AD1
:10790000D3885C1CD4801569EE5C0B4F7E709B1C89
:10791000D380A3B2EB5C3B703B88038000201076E1
:107920000648017006480178552901D0AA21017046
:10793000F0BDC046A401002068110020F510002011
:10794000F4100020B0B50C460546FDF7F9FB3E20CB
:10795000FDF73EFC2846FDF73BFC200AFDF738FC0E
:10796000E0B2FDF735FCFDF713FCB0BD7047002811
:107970000ED0AD21C90000BF491E0A04FBD100BFD3
:1079800000BF00BF00BF00BF00BF401E0104F0D118
:107990007047EFF3108072B6704762B67047000010
:1079A00010B5024601230A48824206D01B4CA2426F
:1079B0000AD19C062030074A01E05C07034A1160A7
:1079C000FBF7D0F90448046010BDC046DC1000206D
:1079D000000C0040E010002000E100E0FBF7B6F9E9
:1079E000FDF7ACFFFDF7FEFFFF204830FDF786FEF8
:1079F0000A480B49FFF7D4FFFAF74AFCF9F7F0FE03
:107A0000084800210180FEF76FF8FBF76FFE06487B
:107A10002021F9F7D0FEFEF7A7FCFCE7200C004080
:107A2000853500085A110020000801400FB410B538
:107A300004A9074B02AA039800F032F8044602A9F1
:107A4000002000F09BF9204610BC08BC04B0184789
:107A50007D7D00082021020C01D010211046020A71
:107A600001D010460839020901D01046091F8208CA
:107A700001D01046891E420801D0881E7047081A9E
:107A8000704702E008C8121F08C1002AFAD17047E7
:107A90007047002001E001C1121F002AFBD170478E
:107AA000FFB58FB00F460446002606E025280AD011
:107AB000129A11999047641C761C20780028F5D101
:107AC000304613B0F0BD00250121A14A009500E029
:107AD0000543641C23780846203B98401042F7D1A8
:107AE00020782E2815D1042005436078641C2A28AC
:107AF0000AD101CF641C00900BE000990A22514387
:107B000030394018641C009020780146303909292A
:107B1000F3D920786C280ED004DC4C2813D06A28C6
:107B200012D104E074280ED07A280DD10BE0012088
:107B30004005054307E00121090562780D438242B3
:107B400001D16D18641C641C2078864669284AD0CF
:107B500008DC0028B4D058286DD0632810D06428E1
:107B600008D140E070286BD0732812D0752860D0FF
:107B7000782860D0129A704611999047761CE5E0FB
:107B80003878694608720020487202A801900120E6
:107B900003E0386801900020C0433F1D69070CD501
:107BA000002500E06D1C00998D420FDA8542F9DB5B
:107BB0000199495D0029F5D108E0002500E06D1C20
:107BC0008542FCDB0199495D0029F8D1761907E06F
:107BD000019801990078491C0191129A11999047D6
:107BE0006D1EF5D2B2E00A20029000216802400F1B
:107BF000039102280CD001CFC117844600290DDA69
:107C00006246084652420021814194462D2008E0F8
:107C1000FF1DFF08FF0003CF8446EFE7280504D5CA
:107C20002B206A46107401203CE0E8073AD020205F
:107C3000F7E70A2000E0102000210391029007E0FE
:107C40001020029000210420054308200391009099
:107C50006802400F022810D001CF00218446002086
:107C60000D9028071FD5704670280CD0029A10205E
:107C7000039B42401A430CD015E0FF1DFF08FF0094
:107C800003CF8446EBE740206A46107401200D9034
:107C90000CE06046084306D030206A4610747046F7
:107CA000507402200D907046582804D029A00190ED
:107CB0000DA80E900DE02CA0F9E76046039B029AF8
:107CC000F8F716FA019B84469B5C0E9A521E0E92A0
:107CD000137060460843F0D10E9805A9081A2030A9
:107CE0000190680701D5009801E0012000900199FA
:107CF000884203DD01460198081A00E000200025B3
:107D0000009006E004A8129A405D119990476D1CFE
:107D1000761C0D988542F5DB04E0129A302011990B
:107D20009047761C0099481E00900029F5DC08E079
:107D30000E980E990078491C0E91129A119990474D
:107D4000761C0199481E01900029F1DC641CB4E600
:107D50000928010030313233343536373839616221
:107D600063646566000000003031323334353637E5
:107D70003839414243444546000000000A68531C1C
:107D80000B60107070470100020005000200020045
:107D9000030000070E091C1B1215383F363124233F
:107DA0002A2D70777E796C6B6265484F464154533B
:107DB0005A5DE0E7EEE9FCFBF2F5D8DFD6D1C4C3AB
:107DC000CACD90979E998C8B8285A8AFA6A1B4B39B
:107DD000BABDC7C0C9CEDBDCD5D2FFF8F1F6E3E40B
:107DE000EDEAB7B0B9BEABACA5A28F8881869394FB
:107DF0009D9A2720292E3B3C35321F18111603046B
:107E00000D0A5750595E4B4C45426F68616673745A
:107E10007D7A898E878095929B9CB1B6BFB8ADAABA
:107E2000A3A4F9FEF7F0E5E2EBECC1C6CFC8DDDABA
:107E3000D3D4696E676075727B7C51565F584D4A2A
:107E40004344191E171005020B0C21262F283D3A1A
:107E500033344E49404752555C5B7671787F6A6D8A
:107E600064633E39303722252C2B0601080F1A1D7A
:107E70001413AEA9A0A7B2B5BCBB9691989F8A8DEA
:107E80008483DED9D0D7C2C5CCCBE6E1E8EFFAFDDA
:107E9000F4F380813A3B3C3D3E3031323334353669
:107EA00049858685868E8F3F405391920000000061
:107EB00000000000000000000000000000000000C2
:107EC00000004653353030312D48320000001E008E
:107ED0001F00000006000C000B000F00040007004C
:107EE0000F000300040006000A000B000C003230F3
:107EF0003235303930310000FA00770100007D0062
:107F0000EE026B030000000000000000002F0000E4
:107F100000000700070000147F147F1400242A7F4C
:107F20002A120062640813230036495522500000CB
:107F30000503000000001C224100000041221C003B
:107F40000014083E08140008083E0808000000A0BD
:107F500060000008080808080000606000000020B9
:107F600010080402003E5149453E0000427F400097
:107F7000004261514946002141454B31001814121D
:107F80007F10002745454539003C4A4949300001EA
:107F90007109050300364949493600064949291E39
:107FA000000036360000000056360000000814229B
:107FB000410000141414141400004122140800029B
:107FC0000151090600324959513E007C1211127CC0
:107FD000007F49494936003E41414122007F4141ED
:107FE000221C007F49494941007F09090901003EDF
:107FF0004149497A007F0808087F0000417F41001D
:10800000002040413F01007F08142241007F404092
:108010004040007F020C027F007F0408107F003E7A
:108020004141413E007F09090906003E4151215E60
:10803000007F091929460046494949310001017F5D
:108040000101003F4040403F001F2040201F003FF3
:108050004038403F006314081463000708700807A5
:1080600000615149454300007F41410000552A55B8
:108070002A55000041417F00000402010204004033
:108080004040404000000102040000205454547855
:10809000007F484444380038444444200038444475
:1080A000487F00385454541800087E090102001813
:1080B000A4A4A47C007F080404780000447D400050
:1080C000004080847D00007F102844000000417F34
:1080D0004000007C04180478007C08040478003810
:1080E0004444443800FC242424180018242418FC98
:1080F000007C0804040800485454542000043F4401
:108100004020003C4040207C001C2040201C003CC3
:108110004030403C004428102844001CA0A0A07C13
:10812000004464544C44141414141414000000004B
:1081300000000000000000000000FC000000000043
:1081400002000000000C020C020000000000000011
:1081500090D0BCD0BC900003000300001824FE4463
:108160008C000302070201001824D8B04C800003E1
:1081700000010201C038E438E000010202010202FD
:10818000080600000000000000000000000000F8E9
:108190000402000000010204000204F800000004D0
:1081A000020100009060F8609000000001000000F3
:1081B0002020FC2020000000010000000000000042
:1081C0000000080600000000202020202000000001
:1081D000000000000000000000000002000000009D
:1081E0000080601C0200040300000000F804040486
:1081F000F8000102020201000008FC000000000279
:108200000302000018844424180003020202020042
:1082100008042424D80001020202010040B088FCB6
:1082200080000000000302003C242424C40001025A
:1082300002020100F824242CC00001020202010005
:108240000C04E41C0400000003000000D8242424D3
:10825000D80001020202010038444444F80000033F
:1082600002020100000010000000000002000000F7
:1082700000002000000000000600000000205088E0
:108280000402000000000102909090909000000015
:1082900000000000000204885020000201000000DD
:1082A0001804C4241800000002000000F804E4943C
:1082B000F80001020202020000E09CF080000203CC
:1082C0000000030204FC2424D8000203020201007F
:1082D000F80404040C0001020202010004FC04047E
:1082E000F80002030202010004FC24740C000203E3
:1082F0000202030004FC24740C00020302000000CC
:10830000F0080444CC4000010202010004FC2020DB
:10831000FC040203000003020404FC040400020243
:1083200003020200000404FC040406040403000029
:1083300004FC24D00C0402030200030204FC040029
:108340000000020302020203FC3CC03CFC000300EC
:108350000300030004FC30C4FC0402030200030019
:10836000F8040404F80001020202010004FC2424C1
:108370001800020302000000F8848404F8000102DF
:108380000207050004FC24649800020302000302B3
:10839000182424448C000302020201000C04FC0493
:1083A0000C0000020302000004FC0000FC040001B9
:1083B00002020100047C80E01C04000003000000B5
:1083C0001CE03CE01C00000300030000049C609CD7
:1083D0000400020300030200041CE01C040000026D
:1083E000030200000C84641C040002030202030068
:1083F0000000FE020200000007040400000E30C06E
:108400000000000000010200000202FE0000000463
:108410000407000000040204000000000000000047
:10842000000000000000080808080808000002001A
:1084300000000000000000000040A0A0C0000001FB
:108440000202030204FC2020C0000003020201001B
:1084500000C02020600000010202020000C02024B1
:10846000FC0000010202030200C0A0A0C000000145
:10847000020202000020F824240400020302020089
:108480000040A0A0602000070A0A0A0404FC202083
:10849000C0000203020003020020E400000000020A
:1084A00003020000000020E40000080808070000A4
:1084B00004FC80E020200203020003020404FC000C
:1084C0000000020203020200E020E020C0000300DE
:1084D0000300030020E02020C0000203020003028A
:1084E00000C02020C00000010202010020E0202086
:1084F000C000080F0A02010000C02020E0000001B7
:10850000020A0F0820E040202000020302000000C1
:108510000060A0A020000002020203000020F8205A
:10852000000000000102020020E00020E000000145
:108530000202030220E0208060200000030100000E
:108540006080E08060000003000300002060806025
:10855000200002030003020020E0208060200808C1
:10856000070100000020A0602000000203020200BA
:10857000000020DE0200000000070400000000FFF1
:1085800000000000000F00000002DE2000000004D8
:1085900007000000020102040402000000000000C5
:1085A00000000000000000000000000000000000CB
:1085B000000000F800000000000000333000000060
:1085C00000100C06100C0600000000000000000067
:1085D00040C07840C0784000043F04043F040400D9
:1085E000007088FC08300000001820FF211E0000E9
:1085F000F008F000E018000000211C031E211E00FE
:1086000000F00888700000001E2123241927211083
:1086100010160E0000000000000000000000000026
:10862000000000E0180402000000000718204000CD
:1086300000020418E00000000040201807000000BD
:10864000404080F0804040000202010F0102020021
:10865000000000F0000000000101011F0101010005
:10866000000000000000000080B07000000000006A
:1086700000000000000000000001010101010101F3
:10868000000000000000000000303000000000008A
:10869000000000008060180400601806010000005F
:1086A00000E010080810E000000F102020100F005C
:1086B000001010F8000000000020203F20200000E3
:1086C000007008080888700000302824222130003B
:1086D00000300888884830000018202020110E0043
:1086E0000000C02010F8000000070424243F2400EC
:1086F00000F80888880808000019212020110E00C1
:1087000000E0108888180000000F112020110E00D2
:1087100000380808C83808000000003F00000000CA
:108720000070880808887000001C222121221C008B
:1087300000E010080810E0000000312222110F00B4
:10874000000000C0C0000000000000303000000049
:1087500000000080000000000000806000000000B9
:1087600000008040201008000001020408102000D2
:10877000404040404040400004040404040404001D
:1087800000081020408000000020100804020100B2
:10879000007048080808F0000000003036010000B2
:1087A000C030C828E810E0000718272423140B0065
:1087B0000000C038E0000000203C230202273820DF
:1087C00008F8888888700000203F202020110E00C3
:1087D000C0300808080838000718202020100800BA
:1087E00008F808080810E000203F202020100F00A3
:1087F00008F88888E8081000203F2020232018006F
:1088000008F88888E8081000203F200003000000D6
:10881000C03008080838000007182020221E020077
:1088200008F808000008F808203F210101213F2036
:10883000000808F8080800000020203F2020000061
:1088400000000808F8080800C08080807F00000051
:1088500008F888C028180800203F2001263820008A
:1088600008F8080000000000203F202020203000F1
:1088700008F8F800F8F80800203F003F003F20000B
:1088800008F830C00008F808203F200007183F0013
:10889000E01008080810E0000F10202020100F0042
:1088A00008F808080808F000203F21010101000035
:1088B000E01008080810E0000F18242438504F007A
:1088C00008F8888888887000203F2000030C30203A
:1088D00000708808080838000038202121221C0078
:1088E000180808F8080818000000203F20000000C1
:1088F00008F808000008F808001F202020201F00AA
:108900000878880000C83808000007380E01000009
:10891000F80800F80008F800033C0700073C0300D3
:10892000081868808068180820302C03032C302039
:108930000838C800C83808000000203F20000000A8
:1089400010080808C8380800203826212020180000
:10895000000000FE020202000000007F40404000D4
:10896000000C30C000000000000000010638C0000C
:1089700000020202FE000000004040407F000000B4
:1089800000000402020204000000000000000000D9
:1089900000000000000000008080808080808080D7
:1089A00000020204000000000000000000000000BF
:1089B00000008080808000000019242222223F20B5
:1089C00008F8008080000000003F112020110E00F8
:1089D0000000008080800000000E11202020110087
:1089E000000000808088F800000E112020103F2039
:1089F0000000808080800000001F222222221300BD
:108A0000008080F0888888180020203F2020000007
:108A10000000808080808000006B949494936000BC
:108A200008F8008080800000203F210000203F20C7
:108A300000809898000000000020203F20200000C7
:108A4000000000809898000000C08080807F0000B7
:108A500008F8000080808000203F24022D30200094
:108A6000000808F8000000000020203F202000003F
:108A70008080808080808000203F20003F20003F59
:108A80008080008080800000203F210000203F2067
:108A90000000808080800000001F202020201F0018
:108AA000808000808000000080FFA12020110E0047
:108AB0000000008080808000000E112020A0FF8038
:108AC000808080008080800020203F2120000100E5
:108AD000000080808080800000332424242419003A
:108AE000008080E0808000000000001F2020000047
:108AF0008080000000808000001F202020103F2088
:108B0000808080000080808000010E300806010017
:108B100080800080008080800F300C030C300F00BC
:108B200000808000808080000020312E0E312000E7
:108B3000808080000080808080818E701806010017
:108B400000808080808080000021302C2221300035
:108B500000000000807C020200000000003F404056
:108B600000000000FF00000000000000FF00000007
:108B70000002027C800000000040403F0000000036
:108B800000060101020204040000000000000000D1
:108B900000000000000000000000000000000000D5
:108BA00000000000000000000000000000000000C5
:108BB000000000000000000000F0F0F000000000E5
:108BC0000000000000017F01000000000000000024
:108BD000001C1C1C0000000000008060301C8C6029
:108BE000301C0C000000000000000000000000002D
:108BF000000000000000000000000000000000E095
:108C00000000000000E000000086E69F8686868661
:108C1000E69F860000011F01010101011F01010003
:108C2000000080C06020F820E0C0000000000307C2
:108C30000C18FF70E18100000000070F10107F107A
:108C40000F0700008060206080000000E02000002E
:108C50000F3020309F70DC371030C0000000100E45
:108C600003000718101807000000C02020E0C00013
:108C70000000000080E01F38E88703C43C040000C7
:108C8000070F1810100B070D1010080000808C4CF7
:108C9000380000000000000000000000000000009C
:108CA00000000000000000000000000000000000C4
:108CB00000000000000080E0300804000000000018
:108CC00000FEFF0100000000000000000000030F94
:108CD0001820400000040830E08000000000000080
:108CE0000000000001FFFE0000000000004020180E
:108CF0000F03000000000000000000000000C000A2
:108D000000000000004266663C18FF183C666642A0
:108D10000000000000000300000000000000000050
:108D20000000800000000000001010101010FF1064
:108D300010101010000000000000030000000000F0
:108D40000000000000000000000000000000000023
:108D5000000000000000000000808C4C3800000083
:108D60000000000000000000000000000000000003
:108D70000010101010101010101010000000000053
:108D800000000000000000000000000000000000E3
:108D900000000000000000000000000000000000D3
:108DA00000001C1C1C00000000000000000000006F
:108DB00000000000E0380C000000000080701C0380
:108DC000000000000060380E0100000000000000FC
:108DD000000080C060202060C080000000FEFF0115
:108DE0000000000001FFFE000001070E181010181F
:108DF0000E0701000000808080C0E000000000003D
:108E00000000000000FFFF00000000000000101044
:108E1000101F1F1010100000008040202020206034
:108E2000C080000000030300804020381F070000BE
:108E3000001C1A1918181818181F00000080C020EC
:108E4000202060C080000000000303001010182FD5
:108E5000E780000000070F10101010180F07000027
:108E6000000000000000C0E0F000000000C0B0887A
:108E7000868180FFFF808000000000000010101F2E
:108E80001F1010000000E060606060606060000023
:108E900000003F1008080818F0E0000000070B1061
:108EA0001010101C0F030000000080C04020202084
:108EB000E0C0000000FCFF211008080818F0E000E6
:108EC0000001070C18101010080F03000000C0E08C
:108ED0006060606060E06000000003000000E01877
:108EE0000700000000000000001F1F00000000003D
:108EF0000080C0602020202060C080000087EF2C10
:108F00001818303068CF830000070F0810101010B9
:108F1000180F07000000C0C020202020C0800000E3
:108F2000001F3F604040402010FFFE0000000C1C6E
:108F3000101010080F0300000000000000000000E7
:108F40000000000000000000000E0E0E00000000F7
:108F500000000000001C1C1C0000000000000000BD
:108F6000000000000000000000000000000C0C00E9
:108F70000000000000000000005838000000000061
:108F800000000000000000804020100000001028B9
:108F90004482010000000000000000000000010207
:108FA00004081000000000000000000000000000A5
:108FB0000084848484848484848484000000000089
:108FC00000000000000000000000102040800000B1
:108FD0000000000000000000000001824428100092
:108FE00000001008040201000000000000C0202062
:108FF0001010101030E0C0000003030000F0100853
:109000000C070300000000001C1C1C0000000000F6
:10901000000000C0406020202040C00000FCFF0194
:10902000F00E03C1FE03807F0001070E081111102E
:10903000110904020000000080E0E00000000000D0
:109040000000807C4340477FF880000010181F100C
:1090500000000000131F1C1020E0E02020202060F2
:10906000C080000000FFFF10101010182FE78000D4
:10907000101F1F1010101010180F0700000080C0E4
:10908000402020202060E00000FCFF0100000000E4
:10909000000001000001070E181010100804030062
:1090A00020E0E02020202040C080000000FFFF00E2
:1090B0000000000001FFFE00101F1F101010180814
:1090C0000E07010020E0E02020202020206080000A
:1090D00000FFFF101010107C00000000101F1F1078
:1090E000101010101018060020E0E0202020202092
:1090F0006060800000FFFF101010107C0000010075
:10910000101F1F100000000000000000000080C0C1
:109110006020202040E0000000FCFF0100004040F3
:10912000C0C140400001070E181010100F0F0000C2
:1091300020E0E0200000000020E0E02000FFFF1021
:109140001010101010FFFF00101F1F100000000073
:10915000101F1F100000202020E0E0202020000031
:109160000000000000FFFF000000000000001010E1
:10917000101F1F101010000000000000202020E031
:10918000E020202000000000000000FFFF000000A1
:109190000060E0808080C07F3F00000020E0E02091
:1091A000000020A06020200000FFFF30187CE3C0FA
:1091B00000000000101F1F10000001131F1C1810DA
:1091C00020E0E020000000000000000000FFFF00A1
:1091D0000000000000000000101F1F1010101010F1
:1091E0001018060020E0E0E000000000E0E0E020D1
:1091F00000FF013FFEC0E01E01FFFF00101F100036
:10920000031F0300101F1F1020E0E0C0000000003B
:109210000020E02000FF0003071C78E08000FF0032
:10922000101F100000000000030F1F00000080C08E
:1092300060202060C080000000FEFF0100000000F0
:1092400000FFFE000001070E181010180C070100A7
:1092500020E0E0202020202060C0800000FFFF20D0
:1092600020202020301F0F00101F1F1000000000C2
:1092700000000000000080C060202060C08000006E
:1092800000FEFF010000000000FFFE000001070ECD
:109290001111133C7C67210020E0E02020202020D9
:1092A00060C0800000FFFF101030F0D0080F0700F2
:1092B000101F1F10000000030F1C10100080C06062
:1092C000202020204040E00000070F0C181830300C
:1092D00060E08100001F0C0810101010180F07002C
:1092E0008060202020E0E02020206080010000003D
:1092F00000FFFF000000000100000000101F1F1011
:109300000000000020E0E020000000000020E0203D
:1093100000FFFF00000000000000FF0000070F1822
:1093200010101010100807002060E0E0200000007E
:1093300020E060200000077FF88000807C030000B0
:1093400000000000071F1C070000000020E0E020D4
:1093500000E0E0200020E0200007FFF8E01FFFFC15
:10936000E01F00000000031F0300011F03000000B6
:10937000002060E0A0000020E0602000000000036A
:109380008F7CF8C6010000000010181E13000117A2
:109390001F1810002060E0E02000000020E06020A6
:1093A000000001073EF8E018070000000000001070
:1093B000101F1F101000000000806020202020A03F
:1093C000E0E0200000000000C0F03E0F03000000BD
:1093D00000101C1F171010101018060000000000CD
:1093E00000FC0404040404000000000000FF00006E
:1093F0000000000000000000007F404040404000AE
:10940000000010E00000000000000000000000006C
:10941000031C60800000000000000000000000034A
:109420000C70800000000404040404FC0000000030
:1094300000000000000000FF0000000000004040AD
:109440004040407F0000000000000010080C040CA9
:1094500008100000000000000000000000000000F4
:1094600000000000000000000000000000000000FC
:1094700000000000000000000000000000000000EC
:1094800000000000808080808080808080808080DC
:1094900000000004040808000000000000000000B4
:1094A00000000000000000000000000000000000BC
:1094B00000000000000000000000000000000000AC
:1094C000000098D844642424FCF80000000F1F1802
:1094D000101010081F1F10180020E0F000000000FE
:1094E000000000000000FFFF180804040CF8F00062
:1094F00000001F0F18101010180F030000000000CC
:10950000000000000000000000E0F8180404043C23
:109510003800000000030F0C1010101008060000A7
:109520000000000000000020E0F0000000E0F81C57
:1095300004040408FFFF000000030F1810101008B7
:109540001F0F0800000000000000000000000000E5
:109550000000E0F8484444444C7870000000030FD9
:109560000C181010100804000000000080C06020DB
:1095700020E0C00000040404FFFF04040404000011
:10958000000010101F1F101010000000000000004D
:109590000000000000000000000070F88C04048C43
:1095A000F874040C007076CF8D8D8D89C8787000AA
:1095B0000020E0F000000000000000000000FFFFBD
:1095C00008040404FCF8000000101F1F1000001025
:1095D0001F1F10000000000000606000000000007D
:1095E0000000040404FCFC00000000000000101057
:1095F000101F1F101010000000000000000000608D
:109600006000000000000000040404FCFC000000F6
:109610000000C0C08080C07F3F0000000020E0F05C
:1096200000000000000000000000FFFF80C0F41CEC
:109630000404000000101F1F1100031F1C10100065
:109640000000202020E0F0000000000000000000EA
:1096500000FFFF000000000000001010101F1F108E
:1096600010100000000000000000000000000000DA
:1096700004FCFC0804FCFC0804FCFC00101F1F1088
:10968000001F1F10001F1F1000000000000000003E
:10969000000000000004FCFC08080404FCF80000C2
:1096A00000101F1F100000101F1F100000000000FE
:1096B000000000000000000000E0F0180C04040CA2
:1096C00018F0E00000030F0C101010100C0F030036
:1096D0000000000000000000000000000004FCFC8E
:1096E000080404040CF8F0000080FFFF88901010BC
:1096F0001C0F03000000000000000000000000003C
:1097000000E0F81C04040408F8FC000000030F1833
:1097100010109088FFFF8000000000000000000093
:1097200000000000040404FCFC100804040C0C00FD
:109730001010101F1F10101000000000000000008B
:10974000000000000000000000003078CCC48484D9
:10975000840C1C0000001E1810101011190F0600B8
:109760000000000000C0000000000000000404042D
:10977000FFFF040404000000000000000F1F101091
:10978000100C0000000000000000000000000000BD
:109790000004FCFE00000004FCFE000000000F1F9F
:1097A000181010081F0F0800000000000000000043
:1097B0000000000000040C3CFCC40000C43C0C048D
:1097C00000000000010F1E0E01000000000000005C
:1097D0000000000000000000043CFCC400E47CFC2D
:1097E00084807C040000071F070000071F0700009B
:1097F0000000000000000000000000000004041C45
:109800007CE4C0341C0404000010101C1601131F5B
:109810001C18100000000000000000000000000004
:1098200000040C3CFCC400C43C0404000000C080E4
:10983000C1370E0100000000000000000000000021
:109840000000000000001C0404C4F47C1C040000A0
:109850000000101C1F17111010180E00000000004F
:10986000000000F80C04000000000000001028EFC9
:1098700000000000000000000000003F6040000009
:10988000000000000000FF000000000000000000D9
:109890000000FF0000000000000000000000FF00CA
:1098A000000000000000040CF800000000000000B0
:1098B00000000000EF2810000000000000004060E1
:1098C0003F0000000000000000180602020408101B
:1098D0002020300800000000000000000000000010
:1098E000000000000000000000000000C0120000A6
:1098F00080250000004B00000096000000E1000001
:1099000000C2010000000000409900080000002093
:1099100020000000827A00086099000820000020E2
:10992000401E0000927A00080000000000000000C5
:109930000000000000000000000000000000000027
:1099400002000102030405060708090A0B000000D3
:109950000024F400010000000000000000000000EE
:04000005080000C12E
:00000001FF
